:100000000C94D2030C94EF030C94B72B0C94EF03D5
:100010000C94EF030C94EF030C94EF030C94EF0398
:100020000C94EF030C9420430C94EF030C94EF0317
:100030000C94EF030C94EF030C94EF030C94EF0378
:100040000C94EF030C94EF030C94EF030C94EF0368
:100050000C94EF030C94B7510C94EF030C94EF0342
:100060000C94EF030C94EF030C94EF030C94EF0348
:100070000C94EF030C94EF030C94EF030C94EF0338
:100080000C94EF030C94EF030C94EF030C94EF0328
:100090000C94EF03A544F044AF45D5454D46714659
:1000A00096469A46AA461F4F1F4F1F4F1F4F1F4F7E
:1000B0001F4F1F4F1F4F1F4F1F4F1F4F1F4F1F4FD0
:1000C0001F4F1F4F1F4F1F4F1F4F1F4F1F4F1F4FC0
:1000D0001F4F3D47BA46D6465B476B47DF4820492E
:1000E000A149E3491F4A924A1F4F1F4F1F4F1F4FFD
:1000F0001F4F1F4F1F4F1F4F1F4F1F4F1F4F1F4F90
:100100001F4F1F4F1F4F1F4F1F4F1F4F1F4F1F4F7F
:100110001F4F9A47DF47004B194B494B604B1F4F0E
:100120001F4F1F4F1F4F1F4F1F4F1F4F1F4F1F4F5F
:100130001F4F0F4867486D4BED4B6C4CAE4C614EFA
:10014000704E254D394D7F4E914EA44E1F4FB54EEA
:100150004C4874489C48E94E044FEF4C0A4D4D4DB5
:10016000814DA44DF04D0B4E364ECE03C103B3036B
:10017000A30390037A036103470329030803E602FC
:10018000C2029E0276024F02280203026C01B801ED
:1001900096017501560139011F010601EF00DA00D1
:1001A000B5008200A5009600000043414E203100BA
:1001B00000000000000000000043414E203200001B
:1001C000000000000000000043414E20330000000A
:1001D0000000000000000043414E203400000000F9
:1001E00000000000000043414E20350000000000E8
:1001F000000000000043414E2036000000000000D7
:100200000000000043414E203700000000000000C5
:1002100000000043414E20380000000000000000B4
:10022000000043414E2039000000000000000000A3
:100230000043414E2031300000000000000000006B
:1002400043414E2031310000000000000000004317
:10025000414E203132000000000000000000434108
:100260004E20313300000000000000000043414EEA
:1002700020313400000000000000000043414E2007
:10028000313500000000000000000043414E2031E5
:100290003600000000000000000043414E203137CE
:1002A00000000000000000000043414E20313800F3
:1002B000000000000000000043414E2031390000E2
:1002C0000000000000000043414E203230000000DA
:1002D00000000000000043414E20323100000000C9
:1002E000000000000043414E2032320000000000B8
:1002F0000000000043414E203233000000000000A7
:1003000000000043414E2032340000000000000095
:10031000000043414E203235000000000000000084
:100320000043414E20323600000000000000000073
:1003300043414E203237000000000000000000431F
:10034000414E203238000000000000000000434110
:100350004E20323900000000000000000043414EF2
:1003600020333000000000000000000043414E2018
:10037000333100000000000000000043414E2033F4
:1003800032000000000000000000466C617368202D
:10039000310000000000000000466C6173682032EC
:1003A0000000000000000000466C6173682033000C
:1003B00000000000000000466C61736820340000FB
:1003C000000000000000466C6173682035000000EA
:1003D00000000000005357495443482031000000FA
:1003E00000000000535749544348203200000000E9
:1003F00000000053574954434820330000000000D8
:1004000000005357495443482034000000000000C6
:1004100000535749544348203500000000000000B5
:100420005357495443482036000000000000005351
:10043000574954434820370000000000000053573C
:100440004954434820380000000000000053574939
:10045000544348203900000000000000535749541D
:1004600043482031300000000000005357495443F6
:10047000482031310000000000004348414E4E4505
:100480004C20310000000000004348414E4E454CD6
:1004900020320000000000004348414E4E454C20F1
:1004A000330000000000004348414E4E454C2034CC
:1004B0000000000000004348414E4E454C203500EE
:1004C00000000000004348414E4E454C20360000DD
:1004D000000000004348414E4E454C2037000000CC
:1004E0000000004348414E4E454C203800000000BB
:1004F00000004348414E4E454C20390000000000AA
:10050000004348414E4E454C203130000000000071
:100510004348414E4E454C2031310000000000431D
:1005200048414E4E454C2031320000000000434807
:10053000414E4E454C2031330000000000434841FD
:100540004E4E454C20313400000000004348414EDF
:100550004E454C20313500000000004348414E4ECE
:10056000454C20313600000000004348414E4E45C6
:100570004C20313700000000004348414E4E454CAE
:1005800020313800000000004348414E4E454C20C9
:10059000313900000000004348414E4E454C2032A6
:1005A0003000000000004348414E4E454C2032319F
:1005B00000000000004348414E4E454C20323200BE
:1005C000000000004348414E4E454C2032330000AD
:1005D0000000004348414E4E454C2032340000009C
:1005E00000004348414E4E454C203235000000008B
:1005F000004348414E4E454C20323600000000007A
:100600004348414E4E454C20323700000000004325
:1006100048414E4E454C203238000000000043480F
:10062000414E4E454C203239000000000043484105
:100630004E4E454C20333000000000004348414EF0
:100640004E454C20333100000000004348414E4EDF
:10065000454C20333200000000004348414E4E45D7
:100660004C20333300000000004348414E4E454CBF
:1006700020333400000000005649525455414C20AC
:10068000310000000000005649525455414C2032C0
:100690000000000000005649525455414C203300E0
:1006A00000000000005649525455414C20340000CF
:1006B000000000005649525455414C2035000000BE
:1006C0000000005649525455414C203600000000AD
:1006D00000005649525455414C203700000000009C
:1006E000005649525455414C20380000000000008B
:1006F0005649525455414C20390000000000005624
:1007000049525455414C20313000000000005649F8
:10071000525455414C2031310000000000564952DE
:100720005455414C203132000000000056495254CB
:1007300055414C20313300000000005649525455B9
:10074000414C2031340000000000564952545541BC
:100750004C20313500000000005649525455414CA0
:1007600020313600000000005649525455414C20BB
:10077000313700000000005649525455414C203199
:100780003800000000005649525455414C20313980
:1007900000000000005649525455414C20323000B0
:1007A0000000000011241FBECFEFD0E1DEBFCDBF9F
:1007B00011E0A0E0B1E0EAEBF7EC00E00BBF02C013
:1007C00007900D92AA3AB107D9F71EE0AAEAB1E064
:1007D00001C01D92A43FB107E1F70C94AB350C9416
:1007E0000000282F277099279695879596958795CD
:1007F0009695879533272330310529F1243031052B
:100800004CF421303105B9F022303105C4F4232BEA
:1008100071F02CC025303105F1F025303105BCF0E8
:1008200026303105E1F027303105E9F01FC0A098EE
:10083000A198A2981BC0A09AA198A29817C0A098AE
:10084000A19AA29813C0A09AA19AA2980FC0A098AA
:10085000A198A29A0BC0A09AA198A29A07C0A098AA
:10086000A19AA29A03C0A09AA19AA29A80628093A8
:100870007C0080917A00806480937A0080917A0075
:1008800084FFFCCF80917A00806180937A00209170
:100890007800809179009927880F991F880F991FF8
:1008A0002295269526952370820F911D0895282F55
:1008B000277099279695879596958795969587950C
:1008C00033272330310529F1243031054CF4213010
:1008D0003105B9F022303105C4F4232B71F02CC05E
:1008E00025303105F1F025303105BCF026303105D9
:1008F000E1F027303105E9F01FC0A098A198A29837
:100900001BC0A09AA198A29817C0A098A19AA298DB
:1009100013C0A09AA19AA2980FC0A098A198A29AD9
:100920000BC0A09AA198A29A07C0A098A19AA29AD7
:1009300003C0A09AA19AA29A806280937C008091C1
:100940007A00806480937A0080917A0084FFFCCFE3
:1009500080917A00806180937A0080917900992754
:10096000089540E050E0FC01029625913491621711
:10097000730760F44B5F5F4FFC0102962591349141
:100980006217730718F446395105A4F3CA01089594
:10099000FC01809100018130B1F410920001F093CC
:1009A000B301E093B201F093B101E093B001F09391
:1009B000AF01E093AE01F093AD01E093AC01F09391
:1009C000AB01E093AA016091B0017091B101709305
:1009D000B3016093B2014091AE015091AF015093C9
:1009E000B1014093B0012091AC013091AD01309341
:1009F000AF012093AE018091AA019091AB01909339
:100A0000AD018093AC01F093AB01E093AA01E80F34
:100A1000F91FE20FF31FE40FF51FCF01860F971F99
:100A200065E070E00E942463CB01089580E10E949C
:100A3000F1030E94C804BC018AE691E00E94B1045F
:100A40009927089583E10E9457049FE4899FC0017C
:100A50001124880F892F881F990B9195A82F8091B9
:100A600001018130C1F4109201018A2F99279093DE
:100A7000BD018093BC019093BB018093BA01909318
:100A8000B9018093B8019093B7018093B601909318
:100A9000B5018093B401E091BA01F091BB01F093EC
:100AA000BD01E093BC016091B8017091B9017093F0
:100AB000BB016093BA014091B6015091B7015093C8
:100AC000B9014093B8012091B4013091B501309340
:100AD000B7012093B6018A2F99279093B50180938F
:100AE000B401820F931F840F951F860F971F8E0FDF
:100AF0009F1F65E070E00E942463862F9927089568
:100B000080E280937C0087E880937A00989A999A93
:100B10009A9AA098A198A298089590E0892F82951A
:100B2000807F8093ED001092EE001092EF00109203
:100B3000F0001092F1001092F2001092F300109267
:100B4000F4001092F5001092F6001092F70080E089
:100B50001092FA008F5F8830D8F39F5F9F30F0F2D9
:100B600008953091ED0090E020EC892F8295807FF0
:100B70008093ED008091EF00822329F43093ED0003
:100B8000892F992708959F5F9F3078F33093ED0068
:100B90008FEF90E008958091EE0086FF03C080E023
:100BA00090E008958091EE0085FF03C081E090E021
:100BB00008958091EF00807C19F48FEF90E0089504
:100BC00082E090E00895BC0140E08091EF00992719
:100BD0008F709070892B89F0FB01E40FF11D8091DB
:100BE000FA0080834F5F242F33278091EF009927ED
:100BF0008F709070281739077CF3089580E89DE086
:100C00000E94F83266E27EE080E00E9435336EEDAD
:100C10007DE081E00E94353368E97DE082E00E945A
:100C2000353381E08093BE018091800D813061F485
:100C30008091810D9091820D6AE070E00E942463A2
:100C400070937E0D60937D0D8091270E813061F44D
:100C50008091280E9091290E6AE070E00E94246332
:100C60007093790D6093780D8091DF0D813061F480
:100C70008091E00D9091E10D6AE070E00E942463A4
:100C800070937C0D60937B0D8091990D813061F4A0
:100C900080919A0D90919B0D6AE070E00E94246310
:100CA0007093250E6093240E0895CF93DF93CDB7F4
:100CB000DEB7CE55D0400FB6F894DEBF0FBECDBF25
:100CC00019828CE0888F84E690E09B838A831D8262
:100CD0001C821E821F82188619861A861B868981AD
:100CE0009E01245F3F4FF901E80FF11D10828F5FD5
:100CF0008C30C8F3CE0101960E94E832A895198E77
:100D00001A8E84E690E09C8F8B8F1E8E1D8E898DAF
:100D10009E012F5F3F4FF901E80FF11D168E8F5F87
:100D20008232C8F3CE0149960E940833A89581E02B
:100D3000898F1A8E84E690E09C8F8B8F1E8E1D8E7D
:100D40008A8D9E012F5F3F4FF901E80FF11D168E2E
:100D50008F5F8232C8F3CE0149960E940833A8956E
:100D600082E0898F1A8E84E690E09C8F8B8F1E8E96
:100D70001D8E8A8D9E012F5F3F4FF901E80FF11DF7
:100D8000168E8F5F8034C8F3CE0149960E940833D7
:100D9000C25ADF4F0FB6F894DEBF0FBECDBFDF9152
:100DA000CF91089599278832910509F440C089327E
:100DB000910594F48532910559F18632910534F408
:100DC00083329105D9F08497F1F04FC086329105B6
:100DD00021F1879739F149C08B329105B9F18C32F5
:100DE000910534F48932910539F18A9751F13DC06A
:100DF0008C32910581F18D9799F137C080EC0E947A
:100E0000EC419927089581EC0E94EC4199270895BF
:100E100082EC0E94EC419927089581ED0E94EC41FB
:100E20009927089584EC0E94EC419927089585EC58
:100E30000E94EC419927089586EC0E94EC41992785
:100E4000089587EC0E94EC419927089583EC0E9455
:100E5000EC419927089582ED0E94EC41992708956D
:100E600083ED0E94EC419927089580E090E0089579
:100E7000EF92FF920F931F93CF93DF93CDB7DEB71F
:100E800065970FB6F894DEBF0FBECDBF8091760E8A
:100E90009091770E01978F5F974008F0ABC39091C8
:100EA000750E992309F4A6C380917A0D8F5F809304
:100EB0007A0D891708F49EC310927A0D88E08D830D
:100EC000FE01369611928A95E9F780917F0D992758
:100ED0008530910509F4AAC2863091059CF48230D0
:100EE000910509F4FEC18330910524F4019709F4BA
:100EF000C1C117C08330910509F42AC2049709F4CF
:100F00005EC20FC08730910509F4E7C287309105B2
:100F10000CF4B8C28930910509F40AC30A9709F4A0
:100F200040C38091760E9091770EAA27BB278983C4
:100F30009A83AB83BC8301E000937F0D10E080ECCB
:100F40000E94EC418111102F81EC0E94EC41811133
:100F5000126082EC0E94EC418111146081ED0E94CC
:100F6000EC418111186084EC0E94EC418111106108
:100F700085EC0E94EC418111106286EC0E94EC41EC
:100F80008111106487EC0E94EC41811110681E836E
:100F900010E083EC0E94EC41811111E082ED0E948F
:100FA000EC418111126083ED0E94EC4181111460CB
:100FB0001F8310E081E090E00E94ED54892B09F03E
:100FC00011E082E090E00E94ED54892B09F012605C
:100FD00083E090E00E94ED54892B09F0146084E0D6
:100FE00090E00E94ED54892B09F0186085E090E0B4
:100FF0000E94ED54892B09F0106186E090E00E9478
:10100000ED54892B09F0106287E090E00E94ED54C6
:10101000892B09F0106488E090E00E94ED54892B40
:1010200009F01068188710E089E090E00E94ED5404
:10103000892B09F011E08AE090E00E94ED54892BA1
:1010400009F012608BE090E00E94ED54892B09F0CA
:1010500014608CE090E00E94ED54892B09F0186038
:101060008DE090E00E94ED54892B09F010618EE034
:1010700090E00E94ED54892B09F010628FE090E01F
:101080000E94ED54892B09F0106480E190E00E94E9
:10109000ED54892B09F01068198710E081E090E089
:1010A0000E94E610892B09F011E082E090E00E9496
:1010B000E610892B09F0126083E090E00E94E610B0
:1010C000892B09F0146084E090E00E94E610892BDF
:1010D00009F0186085E090E00E94E610892B09F085
:1010E000106186E090E00E94E610892B09F0106202
:1010F00087E090E00E94E610892B09F0106488E0F8
:1011000090E00E94E610892B09F010681A8710E021
:1011100089E090E00E94E610892B09F011E08AE056
:1011200090E00E94E610892B09F012608BE090E0BD
:101130000E94E610892B09F014608CE090E00E9478
:10114000E610892B09F018608DE090E00E94E6100F
:10115000892B09F010618EE090E00E94E610892B47
:1011600009F010628FE090E00E94E610892B09F0F0
:10117000106480E190E00E94E610892B09F010686D
:101180001B8710E081E190E00E94E610892B09F0B6
:1011900011E082E190E00E94E610892B09F01260D4
:1011A00083E190E00E94E610892B09F0146084E14D
:1011B00090E00E94E610892B09F0186085E190E02C
:1011C0000E94E610892B09F0106186E190E00E94F0
:1011D000E610892B09F0106287E190E00E94E6108A
:1011E000892B09F0106488E190E00E94E610892BB9
:1011F00009F010681C8710E089E190E00E94E61079
:10120000892B09F011E08AE190E00E94E610892B19
:1012100009F012608BE190E00E94E610892B09F042
:1012200014608CE190E00E94E610892B09F01860B0
:101230008DE190E00E94E610892B09F010618EE1AB
:1012400090E00E94E610892B09F010628FE190E097
:101250000E94E610892B09F0106480E290E00E9461
:10126000E610892B09F010681D87CE0101960E94B7
:101270007B3FC0C18091760E9091770E0196AA2790
:10128000BB2789839A83AB83BC8382E080937F0DE5
:1012900000E00F2EF6E0EF2EFF24F02DEC0EFD1EE9
:1012A000802F8F5F0E94C129FC01878580FF02C0CB
:1012B00014E60BC0878583FF02C015E606C0818156
:1012C000803F11F411E001C010E0F701E00FF11DC3
:1012D00010830F5F083020F3CE0101960E947B3F00
:1012E00089C18091760E9091770E0296AA27BB272E
:1012F00089839A83AB83BC8383E080937F0D00E076
:101300000F2EF6E0EF2EFF24F02DEC0EFD1E802FA9
:10131000875F0E94C129FC01878580FF02C014E617
:101320000BC0878583FF02C015E606C08181803F20
:1013300011F411E001C010E0F701E00FF11D10837E
:101340000F5F083020F3CE0101960E947B3F52C10F
:101350008091760E9091770E0396AA27BB278983FA
:101360009A83AB83BC8384E080937F0D00E00F2ED3
:10137000F6E0EF2EFF24F02DEC0EFD1E802F8F5E89
:101380000E94C129FC01878580FF02C014E60BC0C2
:10139000878583FF02C015E606C08181803F11F476
:1013A00011E001C010E0F701E00FF11D10830F5FA5
:1013B000083020F3CE0101960E947B3F1BC1809133
:1013C000760E9091770E0496AA27BB2789839A837D
:1013D000AB83BC8385E080937F0D00E00F2EF6E0A9
:1013E000EF2EFF24F02DEC0EFD1E802F875E0E9455
:1013F000C129FC01878580FF02C014E60BC08785E8
:1014000083FF02C015E606C08181803F11F411E020
:1014100001C010E0F701E00FF11D10830F5F0830ED
:1014200020F3CE0101960E947B3FE4C08091760EAE
:101430009091770E0596AA27BB2789839A83AB8361
:10144000BC8386E080937F0D00E00F2EF6E0EF2E48
:10145000FF24F02DEC0EFD1E102F1F5F812F0E9428
:10146000C129D701A00FB11DFC01808991899695F2
:1014700087958C93012F183078F3CE0101960E9446
:101480007B3FB8C08091760E9091770E0696AA2782
:10149000BB2789839A83AB83BC8387E080937F0DCE
:1014A00000E00F2EF6E0EF2EFF24F02DEC0EFD1ED7
:1014B000802F875F0E94C129D701A00FB11DFC01B9
:1014C00080899189969587958C930F5F083080F37A
:1014D000CE0101960E947B3F8DC08091760E909147
:1014E000770E0796AA27BB2789839A83AB83BC8391
:1014F00089E080937F0D00E00F2EF6E0EF2EFF24B1
:10150000F02DEC0EFD1E802F8F5E0E94C129D701A9
:10151000A00FB11DFC0180899189969587958C93C8
:101520000F5F023080F3CE0101960E947B3F62C0C4
:101530008091760E9091770E0996AA27BB27898312
:101540009A83AB83BC838AE080937F0DCE010E9695
:101550000E94A7298889282F3327C901880F991F3E
:10156000880F991F880F991F820F931F280F391F0B
:10157000832F99278E832F838989282F332784E609
:1015800090E0289FA001299F500D389F500D1124F5
:10159000852F992788874987CE0101960E947B3F36
:1015A00029C08091760E9091770E0A96AA27BB27C4
:1015B00089839A83AB83BC8310927F0DCE010E96F4
:1015C0000E94A7291E821F82188619868E859F85F4
:1015D0009C01369527953695279536952795892F21
:1015E00099278695869586958A872B87CE010196C1
:1015F0000E947B3F80917D0D90917E0D009709F4B4
:1016000079C0019790937E0D80937D0D892B09F011
:1016100071C08091810D9091820D6AE070E00E940E
:10162000246370937E0D60937D0D8091830D909166
:10163000840DAA27BB2789839A83AB83BC8388E068
:101640008D838091BE018E838091850D0E944B2AEF
:1016500096958795969587958F838091860D0E94A4
:101660004B2A969587959695879588878091870DC3
:101670000E944B2A969587959695879589878091A4
:10168000880D0E944B2A96958795969587958A870F
:101690008091890D0E944B2A9695879596958795FE
:1016A0008B8780918A0D0E944B2A969587959695F7
:1016B00087958C872091BE0180E89DE0FC01E20FB8
:1016C000F11D82850E944B2A969587959695879560
:1016D0008D878091BE01982F9F5F9093BE0180916E
:1016E000970D891718F481E08093BE01CE01019611
:1016F0000E947B3F8091780D9091790D009709F4BD
:1017000005C101979093790D8093780D892B09F08D
:10171000FDC0CE010E960E94A7298091280E9091BF
:10172000290E6AE070E00E9424637093790D609343
:10173000780D80912A0E90912B0EAA27BB278983C2
:101740009A83AB83BC8388E08D83EE240F2EF0E870
:10175000FF2EF02D0E2D802F9927FC01EA5DF14F11
:101760001681133238F4812F0E946129882379F081
:10177000EF280DC01E3238F4812F0E94D206882334
:1017800031F0EF2804C01E3211F4A499EF28F6942A
:101790000F5F083000F3EE82EE240F2EF0E8FF2EEC
:1017A000F02D0E2D802F9927FC01EA5DF14F168553
:1017B000133238F4812F0E946129882379F0EF28B1
:1017C0000DC01E3238F4812F0E94D206882331F0DA
:1017D000EF2804C01E3211F4A499EF28F6940F5F8D
:1017E000083000F3EF82EE240F2EF0E8FF2EF02DEC
:1017F0000E2D802F9927FC01EA5DF14F16891332D7
:1018000038F4812F0E946129882379F0EF280DC0D8
:101810001E3238F4812F0E94D206882331F0EF283F
:1018200004C01E3211F4A499EF28F6940F5F08301B
:1018300000F3E886EE240F2EF0E8FF2EF02D0E2D9B
:10184000802F9927FC01EA5DF14F168D133238F491
:10185000812F0E946129882379F0EF280DC01E3264
:1018600038F4812F0E94D206882331F0EF2804C07B
:101870001E3211F4A499EF28F6940F5F083000F39C
:10188000E986EE2410914C0E133250F4812F0E9401
:101890006129882399F00F2EF0E8EF2EF02D0EC06D
:1018A0001E3240F4812F0E94D206882339F050E87E
:1018B000E52A04C01E3211F4A499EF2810914D0EB0
:1018C000133240F4812F0E946129882389F080E43B
:1018D000E82A0EC01E3240F4812F0E94D2068823CF
:1018E00039F0E0E4EE2A04C01E3211F4A499EF2886
:1018F000EA868E859F856AE070E00E9424636B878C
:101900001C861D86CE0101960E947B3F80917B0D37
:1019100090917C0D009709F4FCC0019790937C0D89
:1019200080937B0D892B09F0F4C08091E00D90919C
:10193000E10D6AE070E00E94246370937C0D609377
:101940007B0D8091E20D9091E30DAA27BB2789833F
:101950009A83AB83BC8388E08D83EE240F2EF0E85E
:10196000FF2EF02D0E2D802F9927FC01E252F24F11
:101970001681133238F4812F0E948729882379F049
:10198000EF280DC01E3238F4812F0E94D206882322
:1019900031F0EF2804C01E3211F4A499EF28F69418
:1019A0000F5F083000F3EE82EE240F2EF0E8FF2EDA
:1019B000F02D0E2D802F9927FC01E252F24F168553
:1019C000133238F4812F0E948729882379F0EF2879
:1019D0000DC01E3238F4812F0E94D206882331F0C8
:1019E000EF2804C01E3211F4A499EF28F6940F5F7B
:1019F000083000F3EF82EE240F2EF0E8FF2EF02DDA
:101A00000E2D802F9927FC01E252F24F16891332D6
:101A100038F4812F0E948729882379F0EF280DC0A0
:101A20001E3238F4812F0E94D206882331F0EF282D
:101A300004C01E3211F4A499EF28F6940F5F083009
:101A400000F3E886EE240F2EF0E8FF2EF02D0E2D89
:101A5000802F9927FC01E252F24F168D133238F491
:101A6000812F0E948729882379F0EF280DC01E322C
:101A700038F4812F0E94D206882331F0EF2804C069
:101A80001E3211F4A499EF28F6940F5F083000F38A
:101A9000E986EE241091040E133250F4812F0E9437
:101AA0008729882399F00F2EF0E8EF2EF02D0EC035
:101AB0001E3240F4812F0E94D206882339F0F0E8CC
:101AC000EF2A04C01E3211F4A499EF281091050EDC
:101AD000133240F4812F0E948729882389F020E463
:101AE000E22A0EC01E3240F4812F0E94D2068823C3
:101AF00039F040E4E42A04C01E3211F4A499EF281E
:101B0000EA8688898B871C861D86CE0101960E94F5
:101B10007B3F8091240E9091250E009709F45CC1C3
:101B200001979093250E8093240E892B09F054C1C0
:101B300080919A0D90919B0D6AE070E00E94246361
:101B40007093250E6093240E80919C0D90919D0DB5
:101B5000AA27BB2789839A83AB83BC8388E08D83C4
:101B6000EE240F2EF0E8FF2EF02D0E2D802F99275A
:101B7000FC01E856F24F1681133238F4812F0E948F
:101B80006129882379F0EF280DC01E3238F4812FA7
:101B90000E94D206882331F0EF2804C01E3211F4CF
:101BA000A499EF28F6940F5F083000F3EE82EE243C
:101BB0000F2EF0E8FF2EF02D0E2D802F9927FC011F
:101BC000E856F24F1685133238F4812F0E946129AE
:101BD000882379F0EF280DC01E3238F4812F0E943F
:101BE000D206882331F0EF2804C01E3211F4A499E4
:101BF000EF28F6940F5F083000F3EF82EE240F2EEB
:101C0000F0E8FF2EF02D0E2D802F9927FC01E856CD
:101C1000F24F1689133238F4812F0E9461298823EC
:101C200079F0EF280DC01E3238F4812F0E94D206C1
:101C3000882331F0EF2804C01E3211F4A499EF2854
:101C4000F6940F5F083000F3E886EE240F2EF0E8DC
:101C5000FF2EF02D0E2D802F9927FC01E856F24F14
:101C6000168D133238F4812F0E946129882379F070
:101C7000EF280DC01E3238F4812F0E94D20688232F
:101C800031F0EF2804C01E3211F4A499EF28F69425
:101C90000F5F083000F3E986EE240F2EF0E8FF2EE8
:101CA000F02D0E2D802F9927FC01E856F24F16A13A
:101CB000133238F4812F0E948729882379F0EF2886
:101CC0000DC01E3238F4812F0E94D206882331F0D5
:101CD000EF2804C01E3211F4A499EF28F6940F5F88
:101CE000083000F3EA86EE240F2EF0E8FF2EF02DE8
:101CF0000E2D802F9927FC01E856F24F16A51332BE
:101D000038F4812F0E948729882379F0EF280DC0AD
:101D10001E3238F4812F0E94D206882331F0EF283A
:101D200004C01E3211F4A499EF28F6940F5F083016
:101D300000F3EB86EE240F2EF0E8FF2EF02D0E2D93
:101D4000802F9927FC01E856F24F16A9133238F478
:101D5000812F0E948729882379F0EF280DC01E3239
:101D600038F4812F0E94D206882331F0EF2804C076
:101D70001E3211F4A499EF28F6940F5F083000F397
:101D8000EC86EE240F2EF0E8FF2EF02D0E2D802F86
:101D90009927FC01EA52F24F1081133238F4812F57
:101DA0000E948729882379F0EF280DC01E3238F46D
:101DB000812F0E94D206882331F0EF2804C01E3202
:101DC00011F4A499EF28F6940F5F083000F3ED8624
:101DD000CE0101960E947B3F65960FB6F894DEBF58
:101DE0000FBECDBFDF91CF911F910F91FF90EF906C
:101DF000089580916C0E90916D0E885E934031F045
:101E000084EF91E090936D0E80936C0E8FE090E0E4
:101E100090936F0E80936E0E89E999E09093710E06
:101E20008093700E1092720E1092730E1092740EB8
:101E30001092750E1092770E1092760EECE6FEE080
:101E4000A0E7B0E08CE090E021E08030920719F448
:101E50000E94D8630895182E0E94D8630895BF92F7
:101E6000CF92DF92EF92FF920F931F93CF93DF9366
:101E7000CDB7DEB7AE970FB6F894DEBF0FBECDBFBD
:101E8000BB24BE016F5F7F4F8B2D0E941E318B2DB7
:101E900099279C0122953295307F3227207F322767
:101EA000B90162537E4F9981492F4170DB018C91BA
:101EB000887F9670842B892B8C930F2EFFEBCF2E6F
:101EC000F1E0DF2EF02DC20ED31E8A819B81F60138
:101ED000918380838C819D81938382834E815F81F6
:101EE000558344838885998597838683D901A9532F
:101EF000BE4F2A858B85982F9295907F822F8F7069
:101F0000892B8C938C8581878D8582878E858387AD
:101F10008F8584878F8D8170982F990F990F990FD6
:101F2000FB018081877F892B808388A1F6018587CB
:101F300089A186878AA18170982F9295907FFB0155
:101F400080818F7E892B80838C918F70833090F578
:101F5000CA01AA2797FDA095BA2FBC01CD010E9406
:101F60003C60DC01CB0128A539A54AA55BA5BC01D5
:101F7000CD010E94565F7B018C018CA5992787FDBE
:101F80009095A92FB92FBC01CD010E943C60DC01C6
:101F9000CB019C01AD01C801B7010E94215FDC01AA
:101FA000CB01BC01CD010E94A25DDC01CB01F60199
:101FB000958384838B2D99279C0122953295307FC0
:101FC0003227207F3227F901E953FE4F8081829525
:101FD0008F708330D8F50F2EFFEBCF2EF1E0DF2E80
:101FE000F02DC20ED31E88859985AA2797FDA0954E
:101FF000BA2FBC01CD010E943C60DC01CB0128A5B9
:1020000039A54AA55BA5BC01CD010E94565F7B01A5
:102010008C018CA5992787FD9095A92FB92FBC011C
:10202000CD010E943C60DC01CB019C01AD01C801E7
:10203000B7010E94215FDC01CB01BC01CD010E94F0
:10204000A25DDC01CB01F601978386832B2D33271C
:10205000C90182959295907F9827807F9827FC01EF
:10206000E253FE4F808186958370813029F4F90117
:10207000E154FC4F808306C08B2D9927FC01E1546D
:10208000FC4F10828B2D9927880F991FFC01E2517C
:10209000FC4F11821082B394FFE1FB1508F0F1CEE2
:1020A000FE01BD96AAEEB8E082E090E021E080302B
:1020B000920719F40E94C76303C0182E0E94C763D9
:1020C0008DA58093EC038EA58093ED031092E00321
:1020D0001092DF03AE960FB6F894DEBF0FBECDBFF1
:1020E000DF91CF911F910F91FF90EF90DF90CF90F4
:1020F000BF9008951F93CF93DF93CDB7DEB7AE9710
:102100000FB6F894DEBF0FBECDBF10E0A895898151
:10211000887F89831B821A821D821C821F821E82F5
:10212000198618861A861B861C8681E08D871E8676
:102130008F871F8E18A219A21AA280E090E0A0E853
:10214000BFE388A799A7AAA7BBA71CA685E0FE01A5
:10215000B39611928A95E9F78FE0FE017096DF0140
:10216000282F1D922A95E9F7189FC0011124865542
:102170009E4FBC01CF010E94C762BE016F5F7F4FBF
:10218000812F0E94E6301F5F103208F4BFCF1EA6D9
:102190001DA6FE01BD96AAEEB8E082E090E021E027
:1021A0008030920719F40E94D86303C0182E0E9451
:1021B000D863AE960FB6F894DEBF0FBECDBFDF91E9
:1021C000CF911F9108958093DF0308950F93CF93CC
:1021D000DF93CDB7DEB721970FB6F894DEBF0FBE01
:1021E000CDBF89838150803270F000E021E0AE01E4
:1021F0004F5F5F4F69E071E082E091E00E94E92C5F
:1022000080E090E007C089819927FC01E254FC4FEF
:102210008081992721960FB6F894DEBF0FBECDBFFF
:10222000DF91CF910F9108958091EC03882381F085
:102230008091ED030E94EC41882351F4482F8FEBED
:1022400093E0FC01E40FF11D10824F5F4032C8F3B0
:1022500040E06EEE73E0AFEBB3E051E0242F3327A4
:10226000C901820F931FFC01E60FF71F8081918146
:10227000009709F1019791838083892BE1F4C901CB
:1022800082959295907F9827807F9827FC01E25352
:10229000FE4F80818695837099278130910539F0B2
:1022A000029749F0F901EA0FFB1F108204C0FD01FB
:1022B000E40FF11D50834F5F403280F2089580910A
:1022C000DF03882399F08091E003882379F080EE82
:1022D00093E0AC014C5F5F4F6091E3038091E103B9
:1022E0009091E2030E94654F1092E00308958F924F
:1022F0009F92AF92BF92CF92DF92EF92FF920F9395
:102300001F93CF93DF938C01EE24FF2499248091B7
:10231000EC03882339F08091ED030E94EC4188237F
:1023200009F432C28091700E9091710E9C01442785
:102330005527F80180819181A281B381821793078B
:10234000A407B50799F48091720EE80FF11D8581FD
:102350009091730E8923891749F40E94FE500E94C0
:102360001F201092890E82E28093120160E070912A
:10237000DF030F2EFFEBAF2EF3E0BF2EF02D8824EE
:102380008394C0906E0ED0906F0E862F9927829501
:102390009295907F9827807F9827EC01C154DE4F5B
:1023A00088819981AA2797FDA095BA2FF8012081ED
:1023B00031814281538182179307A407B50759F0F1
:1023C0008A819B81AA2797FDA095BA2F8217930730
:1023D000A407B507C1F4462F5527CA01840F951FDE
:1023E000FC01E251FC4FD182C082872F733048F04C
:1023F00099279C012F733070CA010396281739075B
:1024000011F4992493948F8583FF09C08D85F80179
:10241000E80FF11D9E858581981709F062C128811A
:1024200039812115310509F45CC1442737FD4095F8
:10243000542FF80180819181A281B3812817390737
:102440004A075B0709F09DC091E08985882379F0F0
:10245000E80FF11D8481E82EFF24FE2CEE248A85EE
:10246000F801E80FF11D8481E80EF11C14C08A8583
:10247000882381F0F801E80FF11D8481E82EFF2404
:102480008F8584FF08C0EE2034F420E03FEFE22A7D
:10249000F32A01C090E0992309F473C088858F70F6
:1024A000992782309105B9F1833091052CF400977A
:1024B00079F00197C1F065C08430910509F44DC0F1
:1024C000843091050CF43EC0059709F451C059C001
:1024D0008C819D818E159F0509F053C0F501E60F93
:1024E000F11D80824EC08F8584FF0BC08C819D8141
:1024F0008E159F050CF045C0F501E60FF11D808299
:1025000040C08C819D818E159F05D8F5F501E60FA1
:10251000F11D808236C08F8584FF0AC08C819D8129
:10252000E816F90674F5F501E60FF11D808229C061
:102530008C819D81E816F90620F5F501E60FF11D65
:1025400080821FC08C819D818E219F21892BC9F0A3
:10255000F501E60FF11D808214C08C819D818E21D2
:102560009F21892B71F4F501E60FF11D808209C0CE
:102570008C819D818E159F0521F0F501E60FF11DDF
:1025800080828A819B819C01442737FD4095542F8E
:10259000F80180819181A281B381281739074A0708
:1025A0005B0709F09EC091E08B85882379F0E80FE6
:1025B000F11D8481E82EFF24FE2CEE248C85F80189
:1025C000E80FF11D8481E80EF11C14C08C8588236E
:1025D00081F0F801E80FF11D8481E82EFF248F853A
:1025E00084FF08C0EE2034F420E03FEFE22AF32A13
:1025F00001C090E0992309F474C0888582958F709A
:10260000992782309105B9F1833091052CF4009718
:1026100079F00197C1F065C08430910509F44DC08F
:10262000843091050CF43EC0059709F451C059C09F
:102630008E819F818E159F0509F053C0F501E60F2D
:10264000F11D10824EC08F8584FF0BC08E819F814B
:102650008E159F050CF045C0F501E60FF11D1082A7
:1026600040C08E819F818E159F05D8F5F501E60F3C
:10267000F11D108236C08F8584FF0AC08E819F8134
:10268000E816F90674F5F501E60FF11D108229C070
:102690008E819F81E816F90620F5F501E60FF11D00
:1026A00010821FC08E819F818E219F21892BC9F0AE
:1026B000F501E60FF11D108214C08E819F818E21DD
:1026C0009F21892B71F4F501E60FF11D108209C0DD
:1026D0008E819F818E159F0521F0F501E60FF11D7A
:1026E00010826F5F603208F450CE8091DF03882340
:1026F00009F44AC0992019F4823009F045C080914C
:10270000E003823009F440C08091E1039091E2033C
:102710009C0144275527F80180819181A281B381D2
:10272000281739074A075B0799F49091E3038481DE
:10273000981771F4892F992798012B5F3F4FAC01AF
:10274000B90180EE93E004960E94CE62892BC9F015
:1027500082E08093E003F80124812093E3038081E9
:1027600091819093E2038093E103822F992798014E
:102770002B5F3F4FAC01B90184EE93E00E94DB6216
:1027800003C081E08093E003DF91CF911F910F910F
:10279000FF90EF90DF90CF90BF90AF909F908F9081
:1027A00008950E948D058091D80082608093D800A2
:1027B0000895CF93DF93EC018981833089F4898573
:1027C000882309F403C188818295807F8093ED007E
:1027D0008091EF008F738093EF0018821986F6C006
:1027E0000E94B105982F81E089879F3F09F4EBC0D3
:1027F0009883892F8295807F8093ED001092EE0060
:102800001092EF001092F7001092F6001092F5006F
:102810001092F4001092F00089819927813091057F
:1028200009F46BC0823091051CF4892B29F0C9C0D2
:10283000029709F4BBC0C5C08A8581FF30C08D8175
:10284000982F990F990F990F8C8182958695877093
:10285000890F8093F3008C81982F990F990F990F0E
:102860008B81829586958770890F8093F2008B818A
:10287000982F990F990F990F8A8182958695877065
:10288000890F8093F1008A81880F880F880F8093C9
:10289000F0008091EF0080618093EF0012C08B8187
:1028A000982F9295990F907E8A8186958695869528
:1028B000890F8093F3008A818295880F807E8093B0
:1028C000F20020E08E81181660F48F819885FC015B
:1028D000E20FF11D80818093FA002F5F8E8128170F
:1028E000A0F39091EF008E81892B8093EF0080916F
:1028F000EF0080648093EF0069C08A8581FF35C056
:102900008D81982F990F990F990F8C8182958695BB
:102910008770890F8093F3008C81982F990F990FFE
:10292000990F8B81829586958770890F8093F2002D
:102930008B81982F990F990F990F8A81829586958F
:102940008770890F8093F1008A81880F880F880F24
:102950008093F0008091EF0080618093EF00809180
:10296000F00084608093F00015C08B81982F9295C1
:10297000990F907E8A81869586958695890F80939A
:10298000F3008A818295880F807E8093F20084E034
:102990008093F0009091EF008E81892B8093EF005F
:1029A0008091EF0080648093EF0010C08091EF0071
:1029B0008F738093EF008091EF0080688093EF0029
:1029C00005C0198603C08FEF90E002C080E090E060
:1029D000DF91CF910895CF93DF93EC018985882310
:1029E00019F482E090E082C088818295807F809394
:1029F000ED000E94CB05813009F06CC019868091F2
:102A0000EF008F708E838F8198850E94E3058091FF
:102A1000F000992784709070959587959595879586
:102A2000982F91708A85282F2E7F292B2A878091B5
:102A3000EF0084FF31C0822F82608A878091F3008B
:102A40008695869586958D838091F200982F969530
:102A5000969596958091F3008295880F807E890FD8
:102A60008C838091F100982F9695969596958091FC
:102A7000F2008295880F807E890F8B838091F00011
:102A8000982F9695969596958091F1008295880F4E
:102A9000807E890F8A8316C08A858D7F8A87809180
:102AA000F3008295869587708B838091F200982F32
:102AB0009295969597708091F300880F880F880FF4
:102AC000890F8A838091EF008F738093EF0080E0FD
:102AD00090E00CC0882349F489878091EF008F73C0
:102AE0008093EF0080E090E001C09927DF91CF91C3
:102AF0000895982F8F3F19F481E090E00895805C4D
:102B0000843128F4892F0E94EC4199270895892F58
:102B10008150803228F4892F0E94E6109927089569
:102B2000892F8152843128F4892F0E944655992794
:102B3000089580E090E00895982F8F3F19F481E088
:102B400090E00895805C843128F4892F0E94CB4066
:102B500099270895892F8150803228F4892F0E9467
:102B6000E61099270895892F8152843128F4892FFE
:102B70000E9446559927089580E090E0089580913D
:102B80007A0E0E947915882321F085E08093E70969
:102B900046C080917F0E0E947915882341F0809174
:102BA000800E8093EA0983E08093E70938C0809122
:102BB000790E0E947915882321F084E08093E7093B
:102BC0002EC080917B0E0E947915882369F0809138
:102BD000E709873049F0863039F086E08093E709CD
:102BE0008AE08093E9091BC08091E709853021F4D0
:102BF00082E08093E70913C08091E709833041F4B4
:102C00008091EA09882321F481E08093E70907C0D5
:102C10008091E709843019F481E08093E70980917D
:102C2000E7098150823058F480917C0E0E949C15F7
:102C300090917D0E981719F41092E70917C08091B2
:102C4000E909882399F48091E709863079F4809125
:102C50007C0E0E949C1590917D0E981739F487E0A8
:102C60008093E70980917E0E8093E80982E699E0DF
:102C70000E94412B0E94F91708951F93CF93DF9371
:102C800010E0812F9927EC01C80FD91FFE01EF57E3
:102C9000F14F8081882309F4B4C00E9479158823FC
:102CA00009F4AFC0FE01EE57F14F808183FDB3C040
:102CB00088608083877099278230910539F183304D
:102CC00091051CF4019729F0A6C0039709F452C09E
:102CD000A2C0812F9927880F991FFC01EE57F14F51
:102CE0009081892F82958F70877021F0892F8F783E
:102CF000808391C0812F9927880F991FFC01EE577F
:102D0000F14F80818F788061808385C0812F9927E2
:102D1000880F991FFC01EE57F14F808182958F70CB
:102D200087709927009719F0019769F018C0812FD3
:102D30009927880F991FFC01EE57F14F80818F78FA
:102D40008061808368C0812F9927880F991FFC01BB
:102D5000EE57F14F80818F78806280835CC0812F35
:102D60009927880F991FFC01EE57F14F80818F78CA
:102D7000808351C0812F9927880F991FFC01EE573E
:102D8000F14F808182958F708770992781309105EE
:102D9000A9F0823091051CF4892B21F027C00297FD
:102DA000C9F024C0812F9927880F991FFC01EE5785
:102DB000F14F80818F78806180832DC0812F99278A
:102DC000880F991FFC01EE57F14F80818F78806248
:102DD000808321C0812F9927880F991FFC01EE570E
:102DE000F14F80818F788063808315C0812F992770
:102DF000880F991FFC01EE57F14F80818F788083F7
:102E00000AC0812F9927880F991FFC01EE57F14FB7
:102E10008081877F80831F5F143008F432CF0E9447
:102E2000F3200E94881F0E946E2210E085E2189F06
:102E3000C0011124EC01CB5CDB4F8C899D8900978C
:102E400019F001979D8B8C8B8D859E85009761F085
:102E500001979E878D8799859F3F31F085E0989FE8
:102E6000C00111249B878A872A853B85211531055E
:102E700061F089858F3F49F0C90101979B878A8757
:102E8000892B19F48F8580628F878A8D9B8D00979F
:102E900079F001979B8F8A8F892B51F48F8586FD5E
:102EA00004C0812F8F5F0E94C72F8F8580648F871A
:102EB0008F81882311F081508F831F5F123208F4B5
:102EC000B5CFDF91CF911F9108958091E9098823B3
:102ED00019F081508093E9098091E7098730B9F4AE
:102EE0008091E809882321F081508093E8090FC080
:102EF00080917B0E0E947915882339F086E08093BB
:102F0000E7098AE08093E90902C01092E7098091FD
:102F1000EA09882319F081508093EA09A49B23C011
:102F20002091E4092F3710F4220F01C02FEF809178
:102F3000740E8A30D0F09091780E981710F0921796
:102F400030F48091780E8F5F8093780E0EC0809160
:102F5000890E882351F48F5F8093890E0E94FE5062
:102F60000E941F2002C01092780E90915909809102
:102F700069099817E0F420E049E659E065E270E05D
:102F8000FA01E20FF11D8281823268F49927869F4F
:102F9000F001879FF00D969FF00D1124E75CFB4F29
:102FA0008081816080832F5F2C3050F30895909151
:102FB000590980916A098917D8F420E049E659E057
:102FC00065E270E0FA01E20FF11D8281823268F45D
:102FD0009927869FF001879FF00D969FF00D112491
:102FE000E75CFB4F80818E7F80832F5F2C3050F316
:102FF0000895CF92DF92EF92FF920F931F93CF939A
:10300000DF9380912F04882309F004C1F82E0F2E3E
:10301000FAE0EF2EF02D8EE0F89EC0011124EC01B5
:10302000C256D64F00E08A818F3F11F401E01DC0E7
:103030009A81892F805C843128F4892F0E94EC4189
:10304000082F13C09A81892F8150803228F4892F4C
:103050000E94E610082F09C09A81892F815284317D
:1030600020F4892F0E944655082F898199278130A5
:103070009105C9F1823091051CF4892B29F0C5C056
:10308000029709F4BFC0C1C0013009F0BEC08F81F2
:103090008E9DC00111249C838B8389858E9DC001E8
:1030A00011249E838D8388818460888310E025E2CB
:1030B00030E0FE01E10FF11D82858F3F71F099270D
:1030C000829FA001839F500D929F500D1124FA0101
:1030D000E75CFB4F8081846080831F5F143048F37E
:1030E00081E0898392C08B819C81009709F48DC017
:1030F00001979C838B83892B81F5288122FF17C040
:103100008F818E9DC00111249C838B83822F8B7FA6
:10311000888310E0FE01E10FF11D82858F3F19F0D9
:1031200060E00E9413191F5F1430A0F316C0888559
:103130008E9DC00111249C838B8388818460888349
:1031400010E0FE01E10FF11D82858F3F19F061E073
:103150000E9413191F5F1430A0F38881282F22705A
:1031600081FD28C08D819E81009709F44EC0019792
:103170009E838D83892B09F048C082E08983122FBA
:1031800025E230E0FE01E10FF11D82858F3F71F0F5
:103190009927829FA001839F500D929F500D11246B
:1031A000FA01E75CFB4F80818B7F80831F5F1430C7
:1031B00048F32BC0002349F5102F0F2EF5E2CF2E38
:1031C000DD24F02DFE01E10FF11D22852F3F99F046
:1031D000822F99278C9DA0018D9D500D9C9D500D97
:1031E0001124FA01E75CFB4F80818B7F808361E0D3
:1031F000822F0E9413191C821B821F5F143010F350
:10320000198203C0002309F40983F39454E05F1585
:1032100008F001CFDF91CF911F910F91FF90EF90B8
:10322000DF90CF900895DF92EF92FF920F931F935C
:10323000CF93DF93CDB7DEB721970FB6F894DEBFFB
:103240000FBECDBF8983162FDD24833260F00D2D94
:1032500021E0AE014F5F5F4F69E872E083E191E0EA
:103260000E94E92C4EC0998185E2989F700111243B
:1032700085E394E0E80EF91EF701858D9927807F9C
:103280009070803A910529F40F2EF1E4DF2EF02D95
:1032900018C0F701858D9927807F9070803B91053C
:1032A00029F40F2EF2E4DF2EF02D0BC000E021E018
:1032B000AE014F5F5F4F65E972E083E191E00E94EC
:1032C000E92C112379F483E0F701878380EF818370
:1032D00087858F7B8787858D41A16D2D8F700E949B
:1032E000CF390FC0113069F4F70117828FE0818365
:1032F000878586798787858D41A16D2D8F700E9486
:103300001A3A21960FB6F894DEBF0FBECDBFDF91FB
:10331000CF911F910F91FF90EF90DF90089520E0E3
:1033200047E759E065E270E08170382F330FFA010A
:10333000E20FF11D8181823270F49927869FF0019E
:10334000879FF00D969FF00D1124E75CFB4F808165
:103350008D7F832B80832F5F2E3048F3089520E0EC
:1033600047E759E065E270E08170382F330FFA01CA
:10337000E20FF11D8189823270F49927869FF00156
:10338000879FF00D969FF00D1124E75CFB4F808125
:103390008D7F832B80832F5F2E3048F3089580919B
:1033A0003104909132040895809130049927089552
:1033B000EF92FF921F93CF93DF937A018093690975
:1033C00060936A0910E0C12FDD27F701EC0FFD1FA4
:1033D00080810E94CE27823220F4FE01E759F64F09
:1033E00082831F5F1C3078F3DF91CF911F91FF9094
:1033F000EF9008957F928F929F92AF92BF92CF925B
:10340000DF92EF92FF920F931F93CF93C0E00E9441
:10341000CF290E94BE2A0E94E92A82E699E00E94F2
:10342000362B1092570910925609C0935809C09331
:103430005A09C0935B09C0935C09C0935D0982E19E
:10344000EFE1F9E011928A95E9F741E359E028EBC1
:1034500031E08C2F9927880F991FFC01E40FF51F8D
:1034600031832083CF5FC231A0F3C0E04EE959E041
:103470002EE030E08C2F9927829FB001839F700D42
:10348000929F700D1124FB01E40FF51F118214822D
:10349000138216821582FB01E256F64F808184600A
:1034A0008083CF5FC53030F30E947633803221F4C1
:1034B00087E68093110103C08EE680931101A5E396
:1034C000B4E041E04093350428EC30E03093480408
:1034D0002093470452EA5093520462EB60935304E2
:1034E000109256049FEF909354045093550483E038
:1034F000809357048D010B5D1F4F40935A04FD01CB
:1035000030AF27ABF801558F668F41A3978F0F2EF1
:10351000F7EAEF2EF02DE0A20F2EFFE0BF2EF02DE8
:10352000B2A2FD01E65BFF4F40937F04338B228BF9
:103530000F2EF3EADF2EF02DD58E83EB868F41A37D
:10354000978F90A389E082A3FD01E159FF4F40933B
:10355000A404338B228BE58E0F2EF7EBCF2EF02DAC
:10356000C68E41A3978F90A38BE082A3FD01EC56FA
:10357000FF4F4093C904338B228B11EA158F0F2E16
:10358000F1EBFF2EF02DF68E41A3978F90A38EE0E6
:1035900082A3FD01E754FF4F4093EE04338B228B4F
:1035A00055EA558F05EB068F41A3978F90A38DE0C9
:1035B00082A3C6E0FD01E252FF4F40931305338B17
:1035C000228B60EA658F70EB768F11A2978F50A3E4
:1035D000C2A3FD01ED5FFE4F40933805338B228B74
:1035E000558F068F11A2978F90A384E082A3FD01CF
:1035F000E85DFE4F40935D05338B228B658F768FA0
:1036000041A3978F60A38AE082A3FD01E35BFE4F95
:1036100040938205338B228B758F54EB568F75E068
:1036200071A3978F90A382E182A3FD01EE58FE4F14
:103630004093A705338B228B64EA658F568F41A395
:10364000978FD0A288E082A3FD01E956FE4F4093F8
:10365000CC05338B228B56EA558F86EB868F11A2D1
:10366000978F60A342A3CCE0FD01E454FE4F40934A
:10367000F105338B228B558F868F41A3978F10A333
:10368000C2A3FD01EF51FE4F40931606338B228BF0
:10369000E58EC68E11A2978F90A382E082A3FD01D2
:1036A000EA5FFD4F40933B06338B228B158FF68EDE
:1036B00011A2978F90A387E082A3FD01E55DFD4FE6
:1036C00040936006338B228BF58E068F71A3978F04
:1036D0002B2D3327AD0185E290E0289FB001299F73
:1036E000700D389F700D1124FB01EA0FFB1F9FEF37
:1036F00090A381E182A3FD01E05BFD4F61E0609357
:10370000850628EC30E0338B228BB4EAB58F0F2E80
:10371000F4EBFF2EF02DF68E11A2978F0F2EF6EA06
:10372000EF2EF02DE0A285E082A3FA01EB58FD4FC9
:103730006093AA06338B228B8D2CD58E03EB068FDC
:1037400011A2978F90A312A2FA01E656FD4F70E4E2
:103750007093CF062FEF3FEF338B228B0F2EF7EABC
:10376000DF2EF02DD58EF68E63E061A3E78E90A359
:1037700092A3FA01E154FD4F7093F406338B228B30
:10378000E58E15EB168F61A3E78E90A392A3FA0145
:10379000EC51FD4F70931907338B228BA5EAA58F4F
:1037A0000F2EF6EB7F2EF02D768E61A3D78E90A391
:1037B00092A3FA01E75FFC4F70933E07338B228B95
:1037C000B58FC68E61A3D78E90A392A3FA01E25D56
:1037D000FC4F70936307338B228B80EA858F068FB3
:1037E00061A3A78F90A392A3FA01ED5AFC4F7093A7
:1037F0008807338B228B0F2EF1EABF2EF02DB58E6A
:103800000F2EF2EBAF2EF02DA68E61A3A78F90A303
:1038100092A3FA01E858FC4F7093AD07338B228BCB
:103820000F2EF2EA9F2EF02D958EA1EBA68F61A3AD
:10383000B78F90A392A3FA01E356FC4F7093D2077F
:10384000338B228B858E0F2EF0EBCF2EF02DC68E74
:1038500061A3B78F90A392A3FA01EE53FC4F70932C
:10386000F707338B228B858F068F82E081A3178F1A
:1038700090A392A3FA01E951FC4F70931C08338B7B
:10388000228BB58EA68E81A3178F90A392A3FA01E7
:10389000E45FFB4F70934108338B228B958EA68F8C
:1038A00081A3F78E90A392A3FA01EF5CFB4F709374
:1038B0006608338B228B858EC68E81A3F78E90A3EC
:1038C00092A3FA01EA5AFB4F70938B08338B228B39
:1038D000D58EF68E81A3778E90A392A3FA01E55838
:1038E000FB4F7093B008338B228BE58EFA01E558BD
:1038F000FB4F168F9A01FA01E558FB4F52E051A396
:10390000778E4FEF40A342A3F901E056FB4FA72F5C
:103910007093D5086FEF7FEF738B628B85EA858F8D
:10392000768E51A397EB978F40A342A3F901EB53F7
:10393000FB4FA093FA08738B628BB58F968F51A3C0
:10394000978F40A342A3C0E0B90145E250E02FE0C9
:1039500001E21EE130E18C2F9927849FF001859FC1
:10396000F00D949FF00D1124CF01E60FF71F158A7B
:10397000148ADC01A75CBB4F8C918C7D8C931786DD
:10398000168A218314A213A216861586148613861E
:10399000128611868C918B7F8C93178A17820087F1
:1039A000168335832283118E108E138E128E148E01
:1039B000CF5FC23280F2CF911F910F91FF90EF90B5
:1039C000DF90CF90BF90AF909F908F907F900895A1
:1039D000EFE1F9E082E1DF011D928A95E9F7CF017D
:1039E0000E94A83220E061E379E048EB51E0822FA9
:1039F0009927880F991FFC01E60FF71F5183408319
:103A00002F5F2231A0F381E399E00E94C83208952C
:103A1000AF92BF92CF92DF92EF92FF920F931F93DC
:103A2000CF93DF93CDB7DEB7C35CD0400FB6F89429
:103A3000DEBF0FBECDBF10E00F2EF5E6EF2EFF2448
:103A4000F02DEC0EFD1E212F332785E290E0289FFC
:103A5000A001299F500D389F500D11249A012B5C15
:103A60003B4FF90182899389892F9927D7018C933C
:103A70008289F7018183F9018681F70182831582AA
:103A800014821682F9018581F7018383F90180850B
:103A9000F70187838FE0189FC001112486589B4F40
:103AA000BC01C70108960E94C762F701178A108EF1
:103AB0001F5F612FC7010E94C631A895123218F20C
:103AC0008E0102581F4F84E6D8018C9388E7F801D5
:103AD00081834CE050E06FEF70E0C80102960E94D5
:103AE000E862C8010E9406308E0104571F4FF8019A
:103AF00081EC81934EE050E06FEF70E0CF010E94C7
:103B0000E862F80117868AE0808B4EE050E06FEFA4
:103B100070E0C80141960E94E862C8010E943430FA
:103B2000A89510E00F2EF4E1DF2EF02D7E01089411
:103B3000E11CF11C0FE0D701ED2D1D92EA95E9F78C
:103B4000109FC00111248B529C4FBC01C7010E94E1
:103B5000C762188A1F5FB701812F0E945D321B3038
:103B600050F3A89510E00F2EF5EBAF2EBB24F02DEF
:103B7000AC0EBD1E0F2EFFE0CF2EF02D0F2EFBEA58
:103B8000EF2EFF24F02DEC0EFD1EDD24D3940FEF5D
:103B9000D501EC2D1D92EA95E9F71C9DC001112479
:103BA00086579C4FBC01C7010A960E94C762D70185
:103BB0001C92F70111821282D382D4828AE085831B
:103BC0008081F701E80FF11D06838F5F8430C8F311
:103BD000BE0165557F4F812F0E9474301F5F1530E5
:103BE000B8F2E6E9F9E018E0DF01212F1D922A95ED
:103BF000E9F7CF010E9454300E94B12AA895E9E765
:103C0000FEE0DF011D921A95E9F781E080937D0EB9
:103C10008EE180937E0E82E38093800EAEE6BFE05D
:103C200088E090E021E08030920719F40E94D86388
:103C300003C0182E0E94D8639E012B5E3F4F8CE478
:103C4000D9011D928A95E9F78CE0A1E2B1E0FE016D
:103C50007796482F0D9001924A95E1F7ADE2B1E0D9
:103C6000FE01BA96582F0D9001925A95E1F7A9E3FB
:103C7000B1E0FE01FD96982F0D9001929A95E1F723
:103C8000A5E4B1E0FE01E05BFF4F0D9001928A9543
:103C9000E1F7F901AEE8BFE08CE490E021E080308C
:103CA000920719F40E94D86303C0182E0E94D863AB
:103CB00088E0E1E8FEE011928A95E9F7CD53DF4F05
:103CC0000FB6F894DEBF0FBECDBFDF91CF911F912D
:103CD0000F91FF90EF90DF90CF90BF90AF9008953D
:103CE000CF92DF92EF92FF920F931F93CF93DF93C8
:103CF000CDB7DEB7E4970FB6F894DEBF0FBECDBFE9
:103D000000E0102F1F5F612FCE0101960E940B3241
:103D1000202F332785E290E0289FA001299F500D96
:103D2000389F500D1124FA01EB5CFB4F89819927D4
:103D3000982F88272A81820F911D938B828B8B81EC
:103D40008683888580878C818583888D8487898D0B
:103D500081878D819E81918F808F8F81848F012FAC
:103D6000123278F289E699E00E94243087E799E0E0
:103D70000E9444308FE199E00E94B83281E399E0DB
:103D80000E94D83286E999E00E9464300E94B12AEC
:103D900000E0BE01665E7F4F802F0E94AD30202F75
:103DA00033278EE090E0289FF001299FF00D389F87
:103DB000F00D11249F01E256F64F8A8D582F517055
:103DC0008081482F4C7F8B8D8170982F990F842F85
:103DD000852B892B8083F901E256F64F8C8D8283E7
:103DE0008D8D87838E8D80878F8D8187F901E85532
:103DF000F64F88A199A1AAA1BBA180839183A28338
:103E0000B3830F5F053028F2E9E7FEE0AEE6BFE0DE
:103E100088E090E021E08030920719F40E94C763A7
:103E200003C0182E0E94C76300E073E142E050E037
:103E3000642F0F2EF1E8CF2EFEE0DF2EF02D0F2E97
:103E4000F3E3EF2EFF24F02DEC0EFD1EFE01F396A2
:103E5000079FC0011124DC01A257B04F4115510545
:103E600051F081E04030580719F40E94C76303C045
:103E7000162E0E94C763802F99279C01280F391F97
:103E8000F901EC0DFD1D8BA98083D901AE57B14F0F
:103E9000F7018181982F97708C918078892B8C9372
:103EA0000F5F043098F2E4960FB6F894DEBF0FBEB1
:103EB000CDBFDF91CF911F910F91FF90EF90DF90D9
:103EC000CF900895CF93DF93EC01862F0E94CE27E9
:103ED0008332D8F4282F332785E290E0289FA00171
:103EE000299F500D389F500D1124FA01EB5CFB4FB8
:103EF0008F89848788819927982F88272981820F25
:103F0000911D938B828B8A818683DF91CF91089557
:103F10001F93CF93C0E01C2F90917709892F815078
:103F2000803238F4892F0E94E6108823B1F011E026
:103F300014C090917709892F8152843138F4892FE8
:103F40000E944655882349F011E007C08091770907
:103F50000E94EC41813009F4182F90918609892F35
:103F60008150803220F4892F0E94E6100EC090917B
:103F70008609892F8152843120F4892F0E94465569
:103F800004C0809186090E94EC418E3FF1F081309F
:103F9000B9F48091E509843020F48F5F8093E509BE
:103FA00009C01092E5098091E609882319F0815033
:103FB0008093E6098091E609882359F4C1E009C09D
:103FC000809187098093E60904C0809187098093D6
:103FD000E609113021F4812F0E948F190CC0C130E5
:103FE00021F48C2F0E94AF1906C080E00E948F1927
:103FF00080E00E94AF19CF911F910895FC01848148
:10400000982F986080EF8283878586798787168AC4
:10401000892F8F7D8483848525E0829FC0011124B0
:1040200096878587892B41F481858F3F29F0829F70
:10403000C00111249387828783E0878308951F93AB
:10404000CF93C0E015E2C19FC0011124FC01EB5CDD
:10405000FB4F8785992783FD02C080FF03C0CF01F6
:104060000E94FE1FCF5FC23270F3CF911F9108955F
:1040700099278C33910509F466C08D339105A4F41A
:1040800088339105A1F1893391051CF4C79721F17B
:10409000A7C089339105B1F18A33910509F43DC078
:1040A000CB9709F445C09CC08034910509F477C0D2
:1040B0008134910544F48E33910509F45AC0CF97A9
:1040C0000CF062C04BC08134910509F473C0823496
:1040D000910509F47AC084C08091820E8077803186
:1040E00019F481E090E0089580E090E008958091D7
:1040F000820E8077803219F481E090E0089580E0AC
:1041000090E008958091820E8077803319F481E0E9
:1041100090E0089580E090E008958091840E80778B
:10412000803119F481E090E0089580E090E00895F6
:104130008091840E8077803219F481E090E00895B8
:1041400080E090E008958091840E8077803319F4A8
:1041500081E090E0089580E090E008958091860EDF
:104160008077803119F481E090E0089580E090E05C
:1041700008958091860E8077803219F481E090E076
:10418000089580E090E008958091860E80778033D6
:1041900019F481E090E0089580E090E00895809126
:1041A000880E8077803119F481E090E0089580E0F6
:1041B00090E008958091880E8077803219F481E034
:1041C00090E0089580E090E008958091880E8077D7
:1041D000803319F481E090E0089580E090E0089544
:1041E00080E090E00895FF920F931F93CF93DF93A9
:1041F00010E00F2EFFE0FF2EF02D82E00E94924291
:1042000085E2189FC0011124EC01CB5CDB4F88854F
:10421000882361F48981803F09F0F4C08C81886033
:104220008C838F85867B8F87FA82ECC02885822FCE
:1042300081508032D0F58F85992783FD24C080FD81
:1042400022C0822F0E94E610882341F089818F309E
:1042500009F0D8C0CE010E94FE1FD4C08981803FE2
:1042600009F0D0C089858F3F09F4CCC08A859B8531
:10427000892B09F0C7C08C8188608C838F85867BF1
:104280008F87FA82BFC088850E94E610882309F0D4
:10429000B9C08981803F09F0B5C08C8188608C836A
:1042A0008F85867B8F87FA82ADC02885822F8152C9
:1042B0008431D0F58F85992783FD24C080FD22C0ED
:1042C000822F0E944655882341F089818F3009F062
:1042D00099C0CE010E94FE1F95C08981803F09F0E0
:1042E00091C089858F3F09F48DC08A859B85892B74
:1042F00009F088C08C8188608C838F85867B8F874E
:10430000FA8280C088850E944655882309F07AC0C9
:104310008981803F09F076C08C8188608C838F858D
:10432000867B8F87FA826EC000E08885853371F4C2
:104330009091E709892F8350823020F0913011F05D
:10434000963011F491E01DC090E01BC08885863343
:1043500051F48091E709853011F0823011F491E039
:1043600010C090E00EC09885892F87538C3028F4B8
:10437000892F0E943820982F04C088850E94EC4124
:10438000982F9E3FA9F08885803C21F49130A1F4BC
:10439000092F12C08D81813021F4913011F4092F41
:1043A0000BC08D81803141F4992331F401E004C0C8
:1043B00088858F3F09F401E0002369F089818F30FF
:1043C00009F58F85992783FD1DC080FD1BC0CE0197
:1043D0000E94FE1F17C08981803F31F08F85992789
:1043E00083FD02C080FF0EC089858F3F59F08A850A
:1043F0009B85892B39F48C8188608C838F85867BA3
:104400008F87FA8289818F3079F48F859927897017
:104410009070892B49F480911201811729F482E26E
:10442000809312011092890E1F5F123208F4E5CEBC
:10443000DF91CF911F910F91FF90089560932F040A
:10444000623019F48FEF809355090895CF93DF936D
:10445000EC0188818150823218F080E090E03BC00E
:1044600088810E94CE27282F898199278F30910536
:1044700021F0803F9105A1F02CC0332785E290E028
:10448000289FA001299F500D389F500D1124FA013B
:10449000EB5CFB4F8FE081838785867F878719C020
:1044A000332785E290E0289FA001299F500D389F77
:1044B000500D1124FA01EB5CFB4F80EF818387855F
:1044C000867F8787168AFA01E75CFB4F80818F7DA4
:1044D000808381E090E0DF91CF9108958F929F9249
:1044E000AF92BF92CF92DF92EF92FF920F931F9302
:1044F000CF93DF93CDB7DEB721970FB6F894DEBF29
:104500000FBECDBFBB24B9828B2CAB2C9B2C109241
:10451000570910925609B0925A09B0925C09B092AC
:104520005B090E9422058093590980912F048823FA
:1045300009F07DC2B9828B2D823208F0FAC482E084
:104540000E9492428824998185E2989FC00111249B
:104550000F2EF5E3CF2EF4E0DF2EF02DC80ED91E7E
:10456000F601858D9927807F9070803A910529F416
:104570000F2EF1E4AF2EF02D18C0F601858D99278E
:10458000807F9070803B910529F40F2EF2E4AF2ECE
:10459000F02D0BC000E021E0AE014F5F5F4F66E8F9
:1045A00077E083E191E00E94E92CF601118A108AFC
:1045B000248122FDBCC0808199278130910509F4B6
:1045C0005DC08034910509F0BFC0818199278F308B
:1045D0009105B1F1803F910509F0B6C0822F83703B
:1045E00019F4878585FF09C0F601858D41A16A2DE3
:1045F0008F700E941A3A882410C0F601858596852E
:10460000892B59F4878580FD08C0858D41A16A2DCD
:104610008F700E94CF3988248394F601848183FFB0
:1046200093C0877F848382818F3009F08DC081831E
:10463000858D41A16A2D8F700E941A3A882484C00A
:10464000F601248123FF80C0822F877F84838281AB
:10465000803F09F079C0818385859685892B09F093
:1046600073C0822F837009F06FC0858D41A16A2DC0
:104670008F700E94CF398824839466C0F6018181AF
:1046800099278F309105C1F1803F910509F05CC0F9
:104690008481837019F4878585FF09C0F601858DB3
:1046A00041A16A2D8F700E941A3A882413C0F60126
:1046B00085859685892B71F48785992780FD0AC0A9
:1046C00083FD08C0858D41A16A2D8F700E94CF396E
:1046D00088248394F601848183FF36C0877F848396
:1046E00082818F3089F58183858D41A16A2D8F70FC
:1046F0000E941A3A882428C0F601248123FF24C08E
:10470000822F877F84838281803FF1F48183858536
:104710009685892BC9F4822F8370B1F4858D41A1D0
:104720006A2D8F700E94CF39882483940DC0F601C2
:10473000818199278F30910531F0803F910521F4D7
:104740008824839401C08824F6018181803F09F088
:1047500058C082A18F3F09F454C00E94F1037C012C
:1047600000271127F601F4A2E3A289819927FC0111
:10477000E15EF64F80819927AA27BB278E159F05FA
:10478000A007B10724F0EE24FF2487010AC0898125
:104790009927FC01E15EF64F8081E81AF1080109D2
:1047A0001109F3E0EF16F10401051105CCF0898140
:1047B0009927880F991FFC01EF5CF64F808191814A
:1047C0009C0144275527C801B7010E94F96220EED9
:1047D00031E040E050E00E946D6379018A0103C03E
:1047E000EE24FF248701F601F18AE08A80915609C0
:1047F000909157098E0D9F1D9093570980935609EC
:1048000003C0F601118A108A882039F4F601828DDE
:10481000938D892B11F0138E128EF60187859927BF
:10482000AC014870507083FD70C020893189828945
:10483000938982179307E0F5828D938D892B11F070
:10484000538F428FF601848185FF26C08489958924
:10485000892B09F05AC087858860878780915A091B
:104860008F5F80935A098081813071F4858D41A1D9
:104870006A2D8F700E941A3A8824898180931201D0
:10488000F60186818093E4098981F6016089718946
:104890008F5F0E945C2F39C0F6018481806284831F
:1048A000968185E0989FC0011124958B848B2DC043
:1048B000F60184818F7D8483208D318D2115310512
:1048C00021F18820A1F0808991898217930778F4DB
:1048D000828D938D892BC9F4878586FD16C0948DB2
:1048E00085E0989FC0011124938F828F0EC0F6013E
:1048F000828D938D892B49F020893189808D918D0E
:104900008217930710F4138E128EF601868D992765
:10491000807F9070803A910529F40F2EF1E49F2E4C
:10492000F02D18C0F601868D9927807F9070803B0E
:10493000910529F40F2EF2E49F2EF02D0BC000E01C
:1049400021E0AE014F5F5F4F6EE978E083E191E0D7
:104950000E94E92CF601868D41A1692D8F700E947D
:104960009D3A282FF6018181803F09F043C0878559
:10497000992783FD3FC080FD3DC0909159098091EA
:1049800011018917B8F5F1E08F1691F5222381F511
:10499000F6018781882371F58485882359F58789F5
:1049A0008F3F11F08F5F878BF6018789863010F17A
:1049B00086898F5F868B843158F4858D41A16A2D5D
:1049C0008F700E941A3AF601178A83E0878312C01B
:1049D000F601858D41A16A2D8F700E941A3AF60169
:1049E00087858160878789818F5F0E94942F02C0AD
:1049F000F601178AF601878580FF05C080915C0962
:104A00008F5F80935C09F601878583FF05C08091E5
:104A10005A098F5F80935A09F60187858111B394F3
:104A200089818F5F8983823208F489CD82C2809127
:104A30002F04813009F0B0C119828981482F823258
:104A400008F077C2242F332785E290E0289FB00139
:104A5000299F700D389F700D1124FB01EB5CFB4FFB
:104A600087858F7D878785E2489FC00111240F2E9F
:104A7000F5E3CF2EF4E0DF2EF02DC80ED91EF6019F
:104A8000858D9927807F9070803A910529F40F2EAB
:104A9000F1E4AF2EF02D0CC0F601858D9927807FB3
:104AA0009070803B910521F40F2EF2E4AF2EF02D93
:104AB000F601848182FD4FC0808199278130910564
:104AC00069F18034910509F046C0818199278F30C2
:104AD000910561F0803F9105F1F5858D41A16A2D29
:104AE0008F700E94CF398824839435C08981282F04
:104AF000332785E290E0289FA001299F500D389F21
:104B0000500D1124FA01EB5CFB4F858DF60141A19C
:104B10006A2D8F700E941A3A88241DC0F601818187
:104B200099278F30910561F0803F9105A1F4858D23
:104B300041A16A2D8F700E94CF39882483940BC0C5
:104B4000F601858D41A16A2D8F700E941A3A8FE07F
:104B5000F60181838824F6018181803F09F057C0E6
:104B600082A18F3F09F453C00E94F1037C0100270A
:104B70001127F601F4A2E3A289819927FC01E15EE5
:104B8000F64F80819927AA27BB278E159F05A0077E
:104B9000B10724F0EE24FF2487010AC089819927F8
:104BA000FC01E15EF64F8081E81AF1080109110964
:104BB000F3E0EF16F10401051105CCF08981992786
:104BC000880F991FFC01EF5CF64F808191819C0159
:104BD00044275527C801B7010E94F96220EE31E051
:104BE00040E050E00E946D6379018A0103C0EE2429
:104BF000FF248701F601F18AE08A8091560990919D
:104C000057098E0D9F1D9093570980935609F60101
:104C100020893189828993898217930788F5848155
:104C200085FF22C084899589892B81F587858860D5
:104C3000878780915A098F5F80935A0980818130DC
:104C400059F4858D41A16A2D8F700E941A3A8824EB
:104C50008FE0F601818382838981F6016089718901
:104C60008F5F0E945C2F12C0F60184818062848372
:104C7000968185E0989FC0011124958B848B06C096
:104C8000F60184818F7D8483158A148AF601868DCE
:104C90009927807F9070803A910529F40F2EF1E4D6
:104CA0009F2EF02D0CC0F601868D9927807F907085
:104CB000803B910521F40F2EF2E49F2EF02DF6019A
:104CC000868D41A1692D8F700E949D3A282FF60193
:104CD0008785992783FD42C080FD40C09091590986
:104CE000809111018917D0F5F1E08F16A9F52223E3
:104CF00099F5F6018781882389F58485882371F5E4
:104D00008181803F59F587898F3F11F08F5F878BB5
:104D1000F6018789863010F186898F5F868B843112
:104D200058F4858D41A16A2D8F700E941A3AF601C0
:104D3000178A83E0878312C0F601858D41A16A2D11
:104D40008F700E941A3AF601878581608787898172
:104D50008F5F0E94942F02C0F601178AF6018785A3
:104D600080FF05C080915C098F5F80935C09F6012C
:104D7000878583FF05C080915A098F5F80935A0908
:104D8000F60187858111B39489818F5F8983482FCC
:104D9000823208F457CECDC080912F04823009F0C2
:104DA000C8C019828981982F823208F0C2C085E27A
:104DB000989FC00111240F2EF5E3CF2EF4E0DF2ED3
:104DC000F02DC80ED91EF601858D9927807F907031
:104DD000803A910529F40F2EF1E4AF2EF02D0CC08E
:104DE000F601858D9927807F9070803B910521F495
:104DF0000F2EF2E4AF2EF02D409155094423D1F04F
:104E0000898199279C012F5F3F4F842F992728176D
:104E1000390741F4F601858D41A16A2D8F700E94FA
:104E2000CF390FC0F601858D41A16A2D8F700E9488
:104E30001A3A07C0F601858D41A16A2D8F700E9434
:104E4000CF39F60182A18F3F09F46CC00E94F103B3
:104E50007C0100271127F601F4A2E3A280912E0421
:104E600080FF1CC089819927FC01E15EF64F80819B
:104E70009927AA27BB278E159F05A007B10724F005
:104E8000EE24FF2487010AC089819927FC01E15E95
:104E9000F64F8081E81AF10801091109F3E0EF16D5
:104EA000F1040105110574F180912E0481FF19C0F0
:104EB00089819927880F991FFC01EF5CF64F80814B
:104EC00091819C0144275527C801B7010E94F962CE
:104ED00020EE31E040E050E00E946D6379018A01EC
:104EE00014C0C801B70128EB31E040E050E00E9457
:104EF000F96220EE31E040E050E00E946D637901FC
:104F00008A0103C0EE24FF248701F601F18AE08ABA
:104F100080915609909157098E0D9F1D90935709C6
:104F20008093560989818F5F8983982F823208F494
:104F30003ECFBB2031F4B0925B09B0925C09B092D5
:104F40005D090E941605982F8093580980913004BE
:104F5000891710F490933004209156093091570925
:104F600080913104909132048217930720F430939A
:104F700032042093310421960FB6F894DEBF0FBEA1
:104F8000CDBFDF91CF911F910F91FF90EF90DF90F8
:104F9000CF90BF90AF909F908F90089581509927A8
:104FA0000895CF93DF93EC01862F0E94CE278332A2
:104FB00078F4282F332785E290E0289FA001299FCD
:104FC000500D389F500D1124FA01EB5CFB4FC68346
:104FD000DF91CF910895EF92FF921F93CF937C01C1
:104FE000C0E080EC0E94EC418111C1E081EC0E94A4
:104FF000EC418111C26082EC0E94EC418111C460DD
:1050000081ED0E94EC418111C86084EC0E94EC416A
:105010008111C06185EC0E94EC418111C06286EC77
:105020000E94EC418111C06487EC0E94EC41811127
:10503000C06810E083EC0E94EC41811111E082ED28
:105040000E94EC418111126083ED0E94EC418111BC
:105050001460F701C0831183C0E081E00E94E61074
:105060008111C1E082E00E94E6108111C26083E0FC
:105070000E94E6108111C46084E00E94E610811154
:10508000C86085E00E94E6108111C06186E00E9440
:10509000E6108111C06287E00E94E6108111C064B1
:1050A00088E00E94E6108111C068F701C283C0E069
:1050B00089E00E94E6108111C1E08AE00E94E610BA
:1050C0008111C2608BE00E94E6108111C4608CE007
:1050D0000E94E6108111C8608DE00E94E6108111E7
:1050E000C0618EE00E94E6108111C0628FE00E94D4
:1050F000E6108111C06480E10E94E6108111C06851
:10510000F701C383C0E081E10E94E6108111C1E094
:1051100082E10E94E6108111C26083E10E94E610E4
:105120008111C46084E10E94E6108111C86085E1AC
:105130000E94E6108111C06186E10E94E610811193
:10514000C06287E10E94E6108111C06488E10E947C
:10515000E6108111C068F701C483C0E089E10E94B4
:10516000E6108111C1E08AE10E94E6108111C2605F
:105170008BE10E94E6108111C4608CE10E94E61070
:105180008111C8608DE10E94E6108111C0618EE13D
:105190000E94E6108111C0628FE10E94E610811129
:1051A000C06480E20E94E6108111C068F701C583E7
:1051B000CF911F91FF90EF9008951F93CF93DF93AE
:1051C000182FEB010E94CE27482F833218F080E081
:1051D00090E073C0992725E230E0829FB001839F61
:1051E000700D929F700D1124FB01E75CFB4F208135
:1051F00022FD24C0FB01EB5CFB4F8181803F71F4F9
:1052000085859685892B39F421FD05C020FD03C0D5
:10521000878585FF03C08FE0888335C0242F33271F
:1052200085E290E0289FF001299FF00D389FF00D56
:105230001124EB5CFB4F8181888325C030E0232F54
:105240005EE0259FC0011124DC01A256B64FFD018E
:105250008181813099F490E07FE060EFFD01E90FFA
:10526000F11D8285841739F431E08C9182FF02C0F0
:10527000788301C068839F5F943080F32F5F25306F
:1052800010F43323F1F2242F332785E290E0289F96
:10529000A001299F500D389F500D1124FA01EB5C9D
:1052A000FB4F87858983808991899C838B83812F9C
:1052B0000E94DF2F8A8381E090E0DF91CF911F91E0
:1052C00008950E94CE27833218F080E090E0089580
:1052D000282F332785E290E0289FA001299F500DB9
:1052E000389F500D1124FA01EB5CFB4F8181803F08
:1052F00059F4FA01E75CFB4F208121FD05C020FD38
:1053000003C081E090E0089580E090E008950E945D
:10531000CE27833218F080E090E00895282F3327BD
:1053200085E290E0289FA001299F500D389F500DE5
:105330001124FA01EB5CFB4F2785283011F0213056
:1053400019F481E090E0089580E090E00895FC0178
:1053500080915609909157099183808380915809D3
:10536000828380915909838380915A098483809133
:105370005B09858380915C09868380915D098783C1
:105380000895982F8150823238F485E2989FC001A9
:105390001124805F9B4F089580E090E008959EEF78
:1053A00081B1892381B982B1892382B917B818B82C
:1053B00091EF8AB189238AB98BB189238BB908957A
:1053C0000F930E94CE27282F833168F000E0202F12
:1053D00040E050E063E47BE083E191E00E94E92C4F
:1053E00080E090E007C08FE199E0FC01E20FF11D41
:1053F000808199270F9108950F930E94CE278331C2
:1054000068F000E0202F40E050E061E57BE083E1C0
:1054100091E00E94E92C80E692E212C09927880F61
:10542000991FFC01EF5CF64F2081318184E190E00F
:10543000289FA001299F500D389F500D1124CA01AB
:105440000F9108950F93CF93DF93EB010E94CE2726
:10545000833158F000E0202F40E050E060E67BE030
:1054600083E191E00E94E92C12C0992721E339E001
:10547000880F991FFC01E20FF31FCE0164E170E079
:105480000E94246371836083C9010E94C832DF9146
:10549000CF910F9108950E94CE27833118F080E0BC
:1054A00090E00895282F332785E290E0289FA001FF
:1054B000299F500D389F500D1124FA01EB5CFB4FD2
:1054C0008089918908950E94CE27833118F080E069
:1054D00090E00895282F332785E290E0289FA001CF
:1054E000299F500D389F500D1124FA01EB5CFB4FA2
:1054F00083A194A1089580932E0460935509089583
:105500001F93CF93C0E015E2C19FC0011124FC019D
:10551000EB5CFB4F82A18F3F41F00E94F1032C2FE7
:105520003327F901E15EF64F8083CF5FC23160F32C
:105530008FE199E00E94A832CF911F910895CF93F7
:1055400080912F04833059F083E080932F04C0E0D2
:1055500061E08C2F0E941319CF5FC232C8F3CF9144
:10556000089580919709882341F00E94BE2A0E94E5
:10557000E92A82E699E00E94362B0895259A2D9813
:10558000269A2E988AEA8093800089E18093810090
:10559000109285001092840080E395E0909387003C
:1055A00080938600109289001092880010928B00E0
:1055B00010928A0010928D0010928C0060E070E0D2
:1055C00081E00E94142B60E070E082E00E94142BC6
:1055D00008951092900084E08093910010929500BD
:1055E00010929400109297001092960010929900D9
:1055F0001092980010929B0010929A0010929D00B9
:1056000010929C0010925F0910925E09109261093D
:1056100010926009809169008860809369001092FF
:105620006A00E99AE19A089599278230910581F0FC
:10563000833091051CF4019721F00895039779F0C8
:105640000895872F99278093890060938800089593
:10565000872F992780938B0060938A000895872F66
:10566000992780938D0060938C000895FC0111822E
:1056700010821382128285E090E0958384831682E3
:105680000895EF92FF920F931F93CF93DF93EC0156
:105690008E81982F8F5F8E83963068F060E375E07F
:1056A00081E00E94142B60E375E082E00E94142BDD
:1056B00086E08E8355C08A819B819C0144275527B3
:1056C000888199817C0100271127DA01C90168943A
:1056D00012F8880F991FAA1FBB1F1694D1F7820FCB
:1056E000931FA41FB51F280F391F4A1F5B1FCA0134
:1056F000B90125E830E040E050E00E94F962A801DD
:1057000097010E944B63E901C9018454904086527D
:10571000944010F0C0E3D5E080919709882349F0C8
:105720008091EF04803F29F4BE0181E00E94142B98
:1057300005C060E375E081E00E94142B8091980918
:10574000882349F080911706803F29F4BE0182E04A
:105750000E94142B05C060E375E082E00E94142BC8
:10576000DF91CF911F910F91FF90EF9008951F92BD
:105770000F920FB60F9211242F933F938F939F9305
:1057800080919400282F3327322F22278091950073
:105790009927282B392B8091690099278C7090705C
:1057A0000C97E1F4309363092093620910929400FE
:1057B0001092950080913304909134049093650980
:1057C0008093640910923404109233041092680993
:1057D000809169008B7F8093690010C0809169007F
:1057E00099278C709070089749F430933404209373
:1057F0003304809169008460809369009F918F9148
:105800003F912F910F900FBE0F901F901895CF933F
:10581000DF93CDB7DEB723970FB6F894DEBF0FBE88
:10582000CDBFFE013196A0E8B1E083E090E021E039
:105830008030920719F40E94C76303C0182E0E949B
:10584000C76343E050E061E571E0CE0101960E943C
:10585000EE51882391F00E94472CE1E5F1E0A0E8A9
:10586000B1E083E090E021E08030920719F40E94DB
:10587000D86303C0182E0E94D863279823960FB6CA
:10588000F894DEBF0FBECDBFDF91CF910895CF93C7
:10589000DF93CDB7DEB76E970FB6F894DEBF0FBEBD
:1058A000CDBF84E1FE013B9611928A95E9F740E075
:1058B00064E124E130E0522FFE013B96469FC00197
:1058C0001124DC01AC57BE4F2115310551F081E0A8
:1058D0002030380719F40E94D86303C0152E0E94A7
:1058E000D863A8954F5F483038F31982FE0131968E
:1058F000A3E8B1E081E090E021E08030920719F464
:105900000E94D86303C0182E0E94D8636E960FB60B
:10591000F894DEBF0FBECDBFDF91CF910895CF9336
:10592000DF93CDB7DEB721970FB6F894DEBF0FBE79
:10593000CDBFFE013196A3E8B1E081E090E021E027
:105940008030920719F40E94C76303C0182E0E948A
:10595000C7638981893010F088E08983898199271C
:1059600021960FB6F894DEBF0FBECDBFDF91CF9169
:105970000895CF93DF93CDB7DEB764970FB6F89451
:10598000DEBF0FBECDBF9B01FE01319694E1899F22
:10599000D0011124A059BE4F84E190E041E0803055
:1059A000940719F40E94C76303C0182E0E94C763AE
:1059B00084E1FE013196D90101900D928A95E1F7BB
:1059C00064960FB6F894DEBF0FBECDBFDF91CF91C6
:1059D00008956F927F928F929F92AF92BF92CF92D3
:1059E000DF92EF92FF920F931F93CF93DF93CDB788
:1059F000DEB7A9970FB6F894DEBF0FBECDBF6C011E
:105A00005B013A01022FFE01B996A3E8B1E081E003
:105A100090E021E08030920719F40E94C76303C030
:105A2000182E0E94C76389A5883008F0D4C0992435
:105A3000FE01759684E1DF011D928A95E9F7B601B2
:105A4000CF010E94F262192D89A5981608F05EC058
:105A50000F2EF4E18F2EF02D0F2EF4E1EF2EFF2408
:105A6000F02DFE013196189DC0011124DC01AC57C8
:105A7000BE4FE114F10459F020E0E21621E0F206F5
:105A800019F40E94C76303C01E2C0E94C7638D8552
:105A90009E858A159B0599F546E050E0B601CE013A
:105AA00001960E94EE51882351F5992493948F8595
:105AB0008A3008F090C0890D8F87053008F004E027
:105AC000198A1A8A1B8A1C8A802F9927AC01B30174
:105AD000CE0141960E94DB62FE013196189DD001F5
:105AE0001124AC57BE4F84E190E021E08030920752
:105AF00019F40E94D86303C0182E0E94D8631F5F58
:105B000089A5181718F4992009F4ABCF992009F04A
:105B100052C089A5883008F04EC08F5F89A78CE0FD
:105B2000FE01319611928A95E9F7F6010190002065
:105B3000E9F731972E2F2C192C3008F02BE010E0CC
:105B4000121780F4AE014F5F5F4F812F9927DC0160
:105B5000A40FB51FF601E80FF91F80818C931F5F1A
:105B6000121798F3BE86AD8681E08F87053008F066
:105B700004E0088B198A1A8A1B8A1C8A802F9927AD
:105B8000AC01B301CE0141960E94DB62FE01319669
:105B900099A584E1989FD0011124A059BE4F84E1BA
:105BA00090E021E08030920719F40E94D86303C08E
:105BB000182E0E94D863FE01B996A3E8B1E081E0F7
:105BC00090E021E08030920719F40E94D86303C06E
:105BD000182E0E94D863A9960FB6F894DEBF0FBEA8
:105BE000CDBFDF91CF911F910F91FF90EF90DF908C
:105BF000CF90BF90AF909F908F907F906F900895BF
:105C0000089582E1EAE8FEE011928A95E9F780E1E1
:105C1000ECE9FEE011928A95E9F7EEEBFEE0A8E8E8
:105C2000B0E082E190E021E08030920719F40E9418
:105C3000C76303C0182E0E94C763E0EDFEE0AAE927
:105C4000B0E082E190E021E08030920719F40E94F8
:105C5000C76303C0182E0E94C763E2EEFEE0ACEA01
:105C6000B0E080E190E021E08030920719F40E94DA
:105C7000C76303C0182E0E94C763ECEAFEE0ADEBD9
:105C8000B0E082E190E021E08030920719F40E94B8
:105C9000C76303C0182E0E94C763EBEEF9E0A5E8C6
:105CA000B0E081E090E021E08030920719F40E949A
:105CB000C76303C0182E0E94C763ECEEF9E0A6E8A4
:105CC000B0E082E090E021E08030920719F40E9479
:105CD000C7630895182E0E94C7630895CF93DF937A
:105CE000CDB7DEB762970FB6F894DEBF0FBECDBF5B
:105CF000FE01319682E1DF011D928A95E9F7A8E85D
:105D0000B0E082E190E021E08030920719F40E9437
:105D1000D86303C0182E0E94D863FE013196AAE909
:105D2000B0E082E190E021E08030920719F40E9417
:105D3000D86303C0182E0E94D863FE013196ACEAE6
:105D4000B0E080E190E021E08030920719F40E94F9
:105D5000D86303C0182E0E94D863FE013196ADEBC4
:105D6000B0E082E190E021E08030920719F40E94D7
:105D7000D86303C0182E0E94D8630E94012E629639
:105D80000FB6F894DEBF0FBECDBFDF91CF9108955F
:105D90000E94D419982F8091EB09891790F4909361
:105DA000EB09EBEEF9E0A5E8B0E081E090E021E05E
:105DB0008030920719F40E94D86303C0182E0E9405
:105DC000D8630E94CF199C018091EC099091ED0954
:105DD00082179307A0F43093ED092093EC09ECEEC1
:105DE000F9E0A6E8B0E082E090E021E080309207A0
:105DF00019F40E94D8630895182E0E94D86308955C
:105E00008091EB09992708958091EC099091ED0913
:105E1000089590E04AE85EE0292F3327F901E40F66
:105E2000F51F808180FF17C08E7F8083D901A8571E
:105E3000BF4FF901E254F14F8081082E0E94CC63DC
:105E4000D901A656BF4FF901E053F14F8081082ECA
:105E50000E94CC630895E92FFF27DF01A40FB51F2F
:105E60008C9181FF0CC08D7F8C93DF01A354BF4FB9
:105E7000E455F14F8081082E0E94CC6308959F5F06
:105E8000923150F290E02CE93EE0E92FFF27DF014C
:105E9000A20FB31F8C91813059F41C92DF01A455DD
:105EA000BF4FEE51F14F8081082E0E94CC630895C0
:105EB0009F5F903150F30895282F2150223198F59B
:105EC0008EEB9EE0FC01E20FF11D3081832F9927BC
:105ED000929582958F7089279F7089278F309105C1
:105EE00014F5482F4F5F942F9295907F832F8F70DA
:105EF000890F8083CB0183709070892B11F041E072
:105F000001C040E03327F901E053F14FCB019695F2
:105F1000879596958795840F8083F901E657F14F11
:105F20008081816080830895E82FE150E231C0F4E0
:105F3000FF27DF01A254B14F2C91822F99278F7038
:105F400090700F971CF5822F8F708F5F922F907F2C
:105F5000890F8C93E657F14F80818160808308958B
:105F60008351803198F4E82FFF27DF01AE51B14F04
:105F70002C91822F99278F7090700F973CF4822F6D
:105F80008F5F8C93E456F14F81E0808308958150B8
:105F90008231A0F4E82FFF27DF01A455B14F2C91E7
:105FA000822F99278F7090700F9744F4822F8F5F04
:105FB0008C93E657F14F8081826080830895E82FAB
:105FC000E150E23188F42E2F3327F901E254F14FEA
:105FD0008081882331F4F901E455F14F80818823D1
:105FE00091F081E090E00895282F2351203158F45A
:105FF00082EE9EE0FC01E20FF11D8081882319F002
:1060000081E090E0089580E090E00895CF93DF93E1
:10601000EC01FC0120E532E08EE090E041E08030D0
:10602000940721F4D9010E94D86304C0D901182E25
:106030000E94D863CE010296AC01698188810E94DA
:10604000D819DF91CF910895FC01A0E5B2E08EE070
:1060500090E021E08030920719F40E94C763089510
:10606000182E0E94C7630895FC01A0E6B2E08FE1FC
:1060700090E021E08030920719F40E94D8630895DF
:10608000182E0E94D8630895FC01A0E6B2E08FE1CB
:1060900090E021E08030920719F40E94C7630895D0
:1060A000182E0E94C7630895FC01ACE7BBE088E0AE
:1060B00090E021E08030920719F40E94D86308959F
:1060C000182E0E94D8630895FC01ACE7BBE088E07D
:1060D00090E021E08030920719F40E94C763089590
:1060E000182E0E94C76308950F93CF93DF93CDB707
:1060F000DEB721970FB6F894DEBF0FBECDBF898300
:10610000853060F000E021E0AE014F5F5F4F67E453
:1061100070E085E591E00E94E92C15C0898199E144
:10612000899FC0011124FB01DC01A252B14F89E11A
:1061300090E021E08030920719F40E94D86303C0F8
:10614000182E0E94D86321960FB6F894DEBF0FBEBA
:10615000CDBFDF91CF910F9108950F93CF93DF9330
:10616000CDB7DEB721970FB6F894DEBF0FBECDBF17
:106170008983853060F000E021E0AE014F5F5F4F22
:1061800064E570E085E591E00E94E92C15C0898105
:1061900099E1899FC0011124FB01DC01A252B14F9A
:1061A00089E190E021E08030920719F40E94C763F2
:1061B00003C0182E0E94C76321960FB6F894DEBF65
:1061C0000FBECDBFDF91CF910F9108950F93CF9365
:1061D000DF93CDB7DEB721970FB6F894DEBF0FBEC1
:1061E000CDBF8983803260F000E021E0AE014F5FD7
:1061F0005F4F60E670E085E591E00E94E92C14C0F5
:10620000FB0199818CE2989FD0011124A659BC4FC3
:106210008CE290E021E08030920719F40E94D8636C
:1062200003C0182E0E94D86321960FB6F894DEBFE3
:106230000FBECDBFDF91CF910F9108950F93CF93F4
:10624000DF93CDB7DEB721970FB6F894DEBF0FBE50
:10625000CDBF8983803260F000E021E0AE014F5F66
:106260005F4F6AE670E085E591E00E94E92C14C07A
:10627000FB0199818CE2989FD0011124A659BC4F53
:106280008CE290E021E08030920719F40E94C7630D
:1062900003C0182E0E94C76321960FB6F894DEBF84
:1062A0000FBECDBFDF91CF910F9108950F93CF9384
:1062B000DF93CDB7DEB721970FB6F894DEBF0FBEE0
:1062C000CDBF8983843160F000E021E0AE014F5FF3
:1062D0005F4F64E770E085E591E00E94E92C14C00F
:1062E000FB01998188E1989FD0011124A451B74FF7
:1062F00088E190E021E08030920719F40E94D86391
:1063000003C0182E0E94D86321960FB6F894DEBF02
:106310000FBECDBFDF91CF910F9108950F93CF9313
:10632000DF93CDB7DEB721970FB6F894DEBF0FBE6F
:10633000CDBF8983843160F000E021E0AE014F5F82
:106340005F4F6EE770E085E591E00E94E92C14C094
:10635000FB01998188E1989FD0011124A451B74F86
:1063600088E190E021E08030920719F40E94C76331
:1063700003C0182E0E94C76321960FB6F894DEBFA3
:106380000FBECDBFDF91CF910F910895CF93DF93D3
:10639000CDB7DEB769970FB6F894DEBF0FBECDBF9D
:1063A000FC01862F8150823218F080E090E02AC0F4
:1063B00061508081898381818A8382818B838381FB
:1063C0008C83878188878789888F808D898F848156
:1063D00095819E838D8386818F83DF0118968FE060
:1063E000FE0139960D9001928A95E1F789E1689F47
:1063F000C00111248457944FBC01CE0101960E9424
:106400009732992769960FB6F894DEBF0FBECDBFBD
:10641000DF91CF9108950F931F93CF93DF93CDB763
:10642000DEB769970FB6F894DEBF0FBECDBF8C0103
:10643000962F91509232B0F589E1989FC0011124B6
:106440009E012F5F3F4FDC01A457B44F89E190E0DC
:1064500041E08030940721F4F9010E94C76304C031
:10646000F901182E0E94C7638981F80180838A810F
:1064700081838B8182838C81838388858783888DC8
:10648000878B898D808F8D819E81958384838F8179
:106490008683D80118968FE0FE01399601900D92FF
:1064A0008A95E1F769960FB6F894DEBF0FBECDBFAF
:1064B000DF91CF911F910F91089581508B30C8F4D7
:1064C000FB01A82FBB27CD0182959295907F98273D
:1064D000807F9827DC01A453B54F80E190E021E054
:1064E0008030920719F40E94D8630895182E0E94F4
:1064F000D863089581508B30C8F4FB01A82FBB27C7
:10650000CD0182959295907F9827807F9827DC0116
:10651000A453B54F80E190E021E08030920719F458
:106520000E94C7630895182E0E94C7630895FC0156
:10653000DB0189E190E021E08030920719F40E94AC
:10654000D86303C0182E0E94D86381E090E00895BC
:10655000FC01A0E1B0E082E190E021E08030920710
:1065600019F40E94D8630895182E0E94D8630895E4
:10657000FC01A0E1B0E082E190E021E080309207F0
:1065800019F40E94C7630895182E0E94C7630895E6
:10659000FC01A0E3B0E084E290E021E080309207CB
:1065A00019F40E94D8630895182E0E94D8630895A4
:1065B000FC01A0E3B0E084E290E021E080309207AB
:1065C00019F40E94C7630895182E0E94C7630895A6
:1065D000FC01A0E8B2E088E190E021E08030920781
:1065E00019F40E94D8630895182E0E94D863089564
:1065F000FC01A0E8B2E088E190E021E08030920761
:1066000019F40E94C7630895182E0E94C763089565
:106610000F93FC018081882319F488E992E016C069
:106620008081813019F48EED92E010C0808182303B
:1066300019F484E293E00AC000E021E0AF0167E4CE
:1066400071E085E591E00E94E92C0DC0DC0186E453
:1066500090E021E08030920719F40E94D86303C0D3
:10666000182E0E94D8630F9108950F93CF93DF9354
:10667000CDB7DEB721970FB6F894DEBF0FBECDBF02
:106680008983882319F488E992E018C089818130D0
:1066900019F48EED92E012C08981823019F484E2FF
:1066A00093E00CC000E021E0AE014F5F5F4F60E679
:1066B00071E085E591E00E94E92C0EC0FB01DC0150
:1066C00086E490E021E08030920719F40E94C763CD
:1066D00003C0182E0E94C76321960FB6F894DEBF40
:1066E0000FBECDBFDF91CF910F910895CF93DF9370
:1066F000CDB7DEB760970FB6F894DEBF0FBECDBF43
:10670000FE013196A0E0B0E080E190E021E0803031
:10671000920719F40E94C76303C0182E0E94C76332
:106720008B858F3119F48FE190E008C08B85803222
:1067300019F480E290E002C08FE190E060960FB61D
:10674000F894DEBF0FBECDBFDF91CF9108950F93B8
:106750001F93CF93DF93CDB7DEB76E970FB6F89444
:10676000DEBF0FBECDBFFE013196A0E0B0E084E0F9
:1067700090E021E08030920719F40E94C76303C0C3
:10678000182E0E94C76344E050E069E671E0CE0134
:1067900001960E94EE51882309F44DC08E010F5FCF
:1067A0001F4F8EE1D8011D928A95E9F785E0E9E651
:1067B000F1E0D80101900D928A95E1F71D821E82C9
:1067C0001F82188619861A861B860E94E81CF8010B
:1067D000A0E0B0E080E190E021E08030920719F481
:1067E0000E94D86303C0182E0E94D863FE01319620
:1067F00084E1DF011D928A95E9F7AAEDBFE084E10B
:1068000090E021E08030920719F40E94D86303C021
:10681000182E0E94D863FE013196A0E0B0E084E01B
:1068200090E021E08030920719F40E94D86303C001
:10683000182E0E94D863FE013196A0E3B2E08AE0F0
:1068400090E021E08030920719F40E94C76303C0F2
:10685000182E0E94C7634AE050E065E871E0CE015F
:1068600001960E94EE51882379F10E94081D0E9432
:106870007A100E94C1530E9455060E94F90EFE0133
:1068800031968EE1DF011D928A95E9F7AEE5BFE012
:1068900080E190E021E08030920719F40E94D863F3
:1068A00003C0182E0E94D863E5E8F1E0A0E3B2E04F
:1068B0008AE090E021E08030920719F40E94D863CA
:1068C00003C0182E0E94D863FE013196A0E8B1E003
:1068D00083E090E021E08030920719F40E94C763C2
:1068E00003C0182E0E94C76343E050E06EE671E0DB
:1068F000CE0101960E94EE51882391F00E94472C10
:10690000EEE6F1E0A0E8B1E083E090E021E0803045
:10691000920719F40E94D86303C0182E0E94D8630E
:10692000FE013196A0E8B0E085E090E021E0803003
:10693000920719F40E94C76303C0182E0E94C76310
:1069400045E050E062E771E0CE0101960E94EE5111
:10695000882309F475C0FE0131968EE1DF011D9296
:106960008A95E9F7ACEBB0E081E090E021E080307F
:10697000920719F40E94D86303C0182E0E94D863AE
:10698000FE013196A5E8B0E081E090E021E08030A2
:10699000920719F40E94D86303C0182E0E94D8638E
:1069A000FE013196A6E8B0E082E090E021E0803080
:1069B000920719F40E94D86303C0182E0E94D8636E
:1069C000FE013196A8E8B0E082E190E021E080305D
:1069D000920719F40E94D86303C0182E0E94D8634E
:1069E000FE013196ACEAB0E080E190E021E0803039
:1069F000920719F40E94D86303C0182E0E94D8632E
:106A0000FE013196ADEBB0E082E190E021E0803014
:106A1000920719F40E94D86303C0182E0E94D8630D
:106A2000E2E7F1E0A0E8B0E085E090E021E080302E
:106A3000920719F40E94D86303C0182E0E94D863ED
:106A4000FE013196AAEDBFE089E090E021E08030C0
:106A5000920731F40E94C76306C00E94D86330C019
:106A6000182E0E94C76390E09E012F5F3F4F8981DF
:106A7000181634F5AE014F5F5F4FF901E90FF11DB4
:106A8000808180538A3090F089E0F90111928A95D3
:106A9000E9F7F901AAEDBFE089E090E021E080305C
:106AA0009207D9F2182E0E94D8630AC09F5F9830CF
:106AB00038F49A01FA01E90FF11D80811816ECF201
:106AC000FE013196A3EEBFE089E090E021E0803046
:106AD000920731F40E94C76306C00E94D86330C099
:106AE000182E0E94C76390E09E012F5F3F4F89815F
:106AF000181634F5AE014F5F5F4FF901E90FF11D34
:106B0000808180538A3090F089E0F90111928A9552
:106B1000E9F7F901A3EEBFE089E090E021E08030E1
:106B20009207D9F2182E0E94D8630AC09F5F98304E
:106B300038F49A01FA01E90FF11D80811816ECF280
:106B40006E960FB6F894DEBF0FBECDBFDF91CF912A
:106B50001F910F910895CFEFD0E1DEBFCDBF0E940E
:106B6000E1500E94C9370E94FA190E9480050E94D4
:106B7000F3500E9436430E94072C0E94A733ECE694
:106B8000FEE0A0E7B0E08CE090E021E080309207EA
:106B900019F40E94C76303C0182E0E94C763809136
:106BA0006C0E90916D0E8A3F910531F18B3F9105EE
:106BB00038F48436910561F08D37910599F039C02C
:106BC00021E0843F920711F1885E934049F131C082
:106BD00086E28093E20084E08093E30083E1809387
:106BE000E40027C08EE18093E20084E08093E3001C
:106BF00083E18093E4001DC08EE08093E20084E096
:106C00008093E30083E18093E40013C086E08093E7
:106C1000E20084E08093E30083E18093E40009C014
:106C200082E08093E20084E08093E30083E180933C
:106C3000E4000E942F0F80916E0E90916F0E0597C9
:106C400038F485E090E090936F0E80936E0E0DC047
:106C500080916E0E90916F0E815D974030F080EDC7
:106C600097E090936F0E80936E0E8091700E9091CE
:106C7000710E28E08030920738F08959994021F050
:106C80001092710E1092700E0E94DB3A0E947053A7
:106C90000E94701E0E947D4287E00E94575D78949A
:106CA0000E94484FA89580E00E9492420E94414372
:106CB000FACF1F93162FA398992787709070880F8B
:106CC000991F81640E94EC50812F0E94EC5080E05B
:106CD0000E94EC50A39A99271F9108950F931F9338
:106CE000162F042FA398992787709070880F991FEB
:106CF00080640E94EC50812F0E94EC50802F0E94F3
:106D0000EC50A39A1F910F9108951F93CF93C091B8
:106D1000EE09CC2389F511E01093EE094CE16AE00D
:106D20008C2F0E946E364C2F6C2F8C2F0E946E364B
:106D30004FEF612F8C2F0E946E364C2F62E08C2F0C
:106D40000E946E364C2F63E08C2F0E946E364C2FC3
:106D500064E08C2F0E946E364C2F65E08C2F0E94D1
:106D60006E364C2F6CE08C2F0E946E364C2F6DE0EF
:106D70008C2F0E946E360AC1C091EE09C13089F590
:106D80004CE16AE08C2F0E946E3640E0642F8C2F1D
:106D90000E946E364FEF6C2F8C2F0E946E3640E0B3
:106DA00062E08C2F0E946E3640E063E08C2F0E94E0
:106DB0006E3640E064E08C2F0E946E3640E065E065
:106DC0008C2F0E946E3640E06CE08C2F0E946E3655
:106DD00040E06DE08C2F0E946E3682E08093EE09D9
:106DE000D5C0C091EE09C23089F54CE16AE08C2F24
:106DF0000E946E3640E0642F8C2F0E946E364FEF5B
:106E000061E08C2F0E946E3640E06C2F8C2F0E9428
:106E10006E3640E063E08C2F0E946E3640E064E006
:106E20008C2F0E946E3640E065E08C2F0E946E36FB
:106E300040E06CE08C2F0E946E3640E06DE08C2FBD
:106E40000E946E3683E08093EE09A0C0C091EE09E7
:106E5000C33089F54CE16AE08C2F0E946E3640E029
:106E6000642F8C2F0E946E364FEF61E08C2F0E94B2
:106E70006E3640E062E08C2F0E946E3640E06C2F50
:106E80008C2F0E946E3640E064E08C2F0E946E369C
:106E900040E065E08C2F0E946E3640E06CE08C2F65
:106EA0000E946E3640E06DE08C2F0E946E3684E0CA
:106EB0008093EE096BC0C091EE09C43089F54CE1B6
:106EC0006AE08C2F0E946E364CEF60E08C2F0E949F
:106ED0006E364FEF61E08C2F0E946E3640E062E02C
:106EE0008C2F0E946E3640E063E08C2F0E946E363D
:106EF00040E06C2F8C2F0E946E3640E065E08C2FB6
:106F00000E946E3640E06CE08C2F0E946E3640E0AE
:106F10006DE08C2F0E946E3685E08093EE0936C0BE
:106F2000C091EE09C53081F54CE16AE08C2F0E94DA
:106F30006E3640E0642F8C2F0E946E3640EF61E089
:106F40008C2F0E946E3640E062E08C2F0E946E36DD
:106F500040E063E08C2F0E946E3640E064E08C2FAE
:106F60000E946E3640E06C2F8C2F0E946E3640E0FF
:106F70006CE08C2F0E946E3640E06DE08C2F0E94FA
:106F80006E361092EE0902C01092EE09CF911F9159
:106F900008959B9AA39A4CE16AE080E00E946E36C5
:106FA00040E064E1842F0E946E3640E0642F842F1D
:106FB0000E946E364FEF61E080E00E946E3640E046
:106FC00062E0842F0E946E3640E063E0842F0E94CE
:106FD0006E3640E064E0842F0E946E3640E065E04B
:106FE000842F0E946E3640E06CE0842F0E946E3643
:106FF00040E06DE0842F0E946E364CE16AE081E053
:107000000E946E3640E064E181E00E946E3640E00E
:10701000642F81E00E946E364FEF61E0862F0E9460
:107020006E3640E062E081E00E946E3640E063E050
:1070300081E00E946E3640E064E081E00E946E369E
:1070400040E065E081E00E946E3640E06CE081E067
:107050000E946E3640E06DE081E00E946E364CE1A9
:107060006AE082E00E946E3640E064E182E00E94C5
:107070006E3640E0642F82E00E946E364FEF61E092
:1070800082E00E946E3640E062E0862F0E946E36FB
:1070900040E063E082E00E946E3640E064E082E01F
:1070A0000E946E3640E065E082E00E946E3640E06D
:1070B0006CE082E00E946E3640E06DE082E00E946B
:1070C0006E364CE16AE083E00E946E3640E064E197
:1070D00083E00E946E3640E0642F83E00E946E36AB
:1070E0004FEF61E083E00E946E3640E062E083E0B3
:1070F0000E946E3640E063E0862F0E946E3640E0CC
:1071000064E083E00E946E3640E065E083E00E9428
:107110006E3640E06CE083E00E946E3640E06DE049
:1071200083E00E946E364CE16AE084E00E946E3695
:1071300040E064E184E00E946E364CEF60E084E061
:107140000E946E364FEF61E084E00E946E3640E0B0
:1071500062E084E00E946E3640E063E084E00E94DA
:107160006E3640E064E0862F0E946E3640E065E0B7
:1071700084E00E946E3640E06CE084E00E946E364F
:1071800040E06DE084E00E946E364CE16AE085E00C
:107190000E946E3640E064E185E00E946E3640E079
:1071A00065E185E00E946E3640E0642F85E00E9434
:1071B0006E3640EF61E085E00E946E3640E062E0AE
:1071C00085E00E946E3640E063E085E00E946E3606
:1071D00040E064E085E00E946E3640E065E0862F86
:1071E0000E946E3640E06CE085E00E946E3640E022
:1071F0006DE085E00E946E3608950F931F93CF9344
:10720000082FC62F142F20E030E0613611F421E062
:1072100030E080E090E0C13411F481E090E0822B16
:10722000932B892B91F060E0812F0E94593621E049
:1072300030E0002E02C0220F331F0A94E2F7482FDD
:10724000422B60E0812F0E946E3620E030E0C23693
:1072500011F421E030E080E090E0C23411F481E0EC
:1072600090E0822B932B892B89F061E0812F0E9483
:10727000593621E030E002C0220F331F0A95E2F7B1
:10728000482F422B61E0812F0E946E36CF911F91D3
:107290000F9108950F931F93CF93082FC62F142F8C
:1072A00020E030E0613611F421E030E080E090E051
:1072B000C13411F481E090E0822B932B892BA1F053
:1072C00060E0812F0E94593621E030E0002E02C09C
:1072D000220F331F0A94E2F7922F9095482F4923EB
:1072E00060E0812F0E946E3620E030E0C23611F45B
:1072F00021E030E080E090E0C23411F481E090E0E1
:10730000822B932B892B99F061E0812F0E945936B3
:1073100021E030E002C0220F331F0A95E2F7922FDE
:107320009095482F492361E0812F0E946E36CF91BE
:107330001F910F9108950F931F93CF93182FC62F6E
:10734000042F20E030E0613611F421E030E080E0ED
:1073500090E0C13411F481E090E0822B932B892BD3
:1073600029F0412F64E1802F0E946E3620E030E04A
:10737000C23611F421E030E080E090E0C23411F434
:1073800081E090E0822B932B892B29F0412F65E13E
:10739000802F0E946E36CF911F910F9108950F9309
:1073A0001F93CF93082FC62F142F50E020E030E01A
:1073B000613611F421E030E080E090E0C13411F456
:1073C00081E090E0822B932B892B71F062E1812F79
:1073D0000E94593621E030E0002E02C0220F331FF8
:1073E0000A94E2F7582F522B20E030E0C23611F415
:1073F00021E030E080E090E0C23411F481E090E0E0
:10740000822B932B892B69F063E1812F0E945936DF
:1074100021E030E002C0220F331F0A95E2F7582F17
:10742000522B412F6C2F852F0E949B39CF911F919A
:107430000F9108950F931F93CF93082FC62F142FEA
:1074400050E020E030E0613611F421E030E080E0EF
:1074500090E0C13411F481E090E0822B932B892BD2
:1074600081F062E1812F0E94593621E030E0002E48
:1074700002C0220F331F0A94E2F7922F9095582FE3
:10748000592320E030E0C23611F421E030E080E002
:1074900090E0C23411F481E090E0822B932B892B91
:1074A00079F063E1812F0E94593621E030E002C07B
:1074B000220F331F0A95E2F7922F9095582F5923E8
:1074C000412F6C2F852F0E949B39CF911F910F91D7
:1074D00008951F93CF93C82F162F40E020E030E08F
:1074E000813611F421E030E080E090E0C13411F405
:1074F00081E090E0822B932B892B29F062E1812F90
:107500000E945936482F20E030E0C23611F421E0C5
:1075100030E080E090E0C23411F481E090E0822B12
:10752000932B892B29F063E1812F0E945936482F34
:10753000842F9927CF911F9108950F931F93CF9375
:10754000182FC62F042F40E020E030E0613611F400
:1075500021E030E080E090E0C13411F481E090E07F
:10756000822B932B892B29F062E1802F0E945936C0
:10757000482F20E030E0C23611F421E030E080E016
:1075800090E0C23411F481E090E0822B932B892BA0
:1075900029F063E1802F0E945936482F81E090E066
:1075A00002C0880F991F1A95E2F784239927CF917B
:1075B0001F910F9108950E94D1138CE49AE090934B
:1075C000E30A8093E20A1092E40A1092DB0A109216
:1075D000DC0A8BED9AE00E94D9138823D1F7109230
:1075E000DA0A84E59AE09093EF0A8093EE0A10920B
:1075F000F00A1092E70A1092E80A87EE9AE00E94D9
:10760000D9138823D1F71092E60A8CE59AE090937B
:10761000FB0A8093FA0A1092FC0A1092F30A109265
:10762000F40A83EF9AE00E94D9138823D1F71092CD
:10763000F20A84E69AE09093070B8093060B10926F
:10764000080B1092FF0A1092000B8FEF9AE00E9435
:10765000D9138823D1F71092FE0A8CEF99E090930A
:10766000740A8093730A1092750A10926C0A82E071
:1076700080936D0A8CE69AE00E94D9138823D1F793
:1076800084E09AE090937F0A80937E0A1092800AA9
:107690001092770A82E08093780A87E79AE00E9446
:1076A000D9138823D1F78CE09AE090938A0A8093CB
:1076B000890A10928B0A1092820A82E08093830AD0
:1076C00082E89AE00E94D9138823D1F784E19AE0F6
:1076D0009093950A8093940A1092960A10928D0ABC
:1076E00082E080938E0A8DE89AE00E94D913882365
:1076F000D1F78CE19AE09093A00A80939F0A1092B0
:10770000A10A1092980A82E08093990A88E99AE087
:107710000E94D9138823D1F784E29AE09093AB0AB0
:107720008093AA0A1092AC0A1092A30A82E0809376
:10773000A40A83EA9AE00E94D9138823D1F78CE245
:107740009AE09093B60A8093B50A1092B70A109205
:10775000AE0A82E08093AF0A8EEA9AE00E94D913C3
:107760008823D1F784E39AE09093C10A8093C00AFA
:107770001092C20A1092B90A82E08093BA0A89EB89
:107780009AE00E94D9138823D1F78CE39AE0909372
:10779000CC0A8093CB0A1092CD0A1092C40A82E0E0
:1077A0008093C50A84EC9AE00E94D9138823D1F70C
:1077B00084E49AE09093D70A8093D60A1092D80A6C
:1077C0001092CF0A82E08093D00A8FEC9AE00E9458
:1077D000D9138823D1F708958091DA0A8823E1F03C
:1077E0008091DA0A813059F48AED9AE001960E947C
:1077F000D913882389F482E08093DA0A0DC080913E
:10780000DA0A823049F48AED9AE001960E94EB147C
:10781000882311F48093DA0A8091E60A8823E1F044
:107820008091E60A813059F486EE9AE001960E9432
:10783000D913882389F482E08093E60A0DC08091F1
:10784000E60A823049F486EE9AE001960E94EB1433
:10785000882311F48093E60A8091F20A8823E1F0EC
:107860008091F20A813059F482EF9AE001960E94E9
:10787000D913882389F482E08093F20A0DC08091A5
:10788000F20A823049F482EF9AE001960E94EB14EA
:10789000882311F48093F20A8091FE0A8823E1F094
:1078A0008091FE0A813059F48EEF9AE001960E9491
:1078B000D913882389F482E08093FE0A0895809189
:1078C000FE0A823049F48EEF9AE001960E94EB1492
:1078D000882311F48093FE0A0895CF93DF93EC017F
:1078E0008CE69AE00E94EB14882309F046C0809150
:1078F0006E0A90916F0AAA27BB2788839983AA836F
:10790000BB83E091730AF091740A80818D83E091CA
:10791000730AF091740A81818E83E091730AF09169
:10792000740A82818F83E091730AF091740A8381D3
:107930008887E091730AF091740A84818987E091C5
:10794000730AF091740A85818A87E091730AF09135
:10795000740A86818B87E091730AF091740A87819B
:107960008C878091720A8C838CE69AE00E94D913EE
:107970008823D1F781E090E0BBC287E79AE00E94BC
:10798000EB14882309F046C08091790A90917A0A15
:10799000AA27BB2788839983AA83BB83E0917E0AA9
:1079A000F0917F0A80818D83E0917E0AF0917F0AB9
:1079B00081818E83E0917E0AF0917F0A82818F839C
:1079C000E0917E0AF0917F0A83818887E0917E0AA8
:1079D000F0917F0A84818987E0917E0AF0917F0A85
:1079E00085818A87E0917E0AF0917F0A86818B8764
:1079F000E0917E0AF0917F0A87818C8780917D0AD1
:107A00008C8387E79AE00E94D9138823D1F781E01D
:107A100090E06EC282E89AE00E94EB14882309F09D
:107A200046C08091840A9091850AAA27BB27888343
:107A30009983AA83BB83E091890AF0918A0A8081A5
:107A40008D83E091890AF0918A0A81818E83E09189
:107A5000890AF0918A0A82818F83E091890AF091E4
:107A60008A0A83818887E091890AF0918A0A848151
:107A70008987E091890AF0918A0A85818A87E09155
:107A8000890AF0918A0A86818B87E091890AF091B0
:107A90008A0A87818C878091880A8C8382E89AE0A1
:107AA0000E94D9138823D1F781E090E021C28DE8AC
:107AB0009AE00E94EB14882309F046C080918F0A57
:107AC0009091900AAA27BB2788839983AA83BB83B6
:107AD000E091940AF091950A80818D83E091940A57
:107AE000F091950A81818E83E091940AF091950A34
:107AF00082818F83E091940AF091950A838188872F
:107B0000E091940AF091950A84818987E091940A22
:107B1000F091950A85818A87E091940AF091950AFF
:107B200086818B87E091940AF091950A87818C87F2
:107B30008091930A8C838DE89AE00E94D913882360
:107B4000D1F781E090E0D4C188E99AE00E94EB147B
:107B5000882309F046C080919A0A90919B0AAA272F
:107B6000BB2788839983AA83BB83E0919F0AF09106
:107B7000A00A80818D83E0919F0AF091A00A818103
:107B80008E83E0919F0AF091A00A82818F83E09119
:107B90009F0AF091A00A83818887E0919F0AF09163
:107BA000A00A84818987E0919F0AF091A00A8581CB
:107BB0008A87E0919F0AF091A00A86818B87E091E5
:107BC0009F0AF091A00A87818C8780919E0A8C83FE
:107BD00088E99AE00E94D9138823D1F781E090E0E8
:107BE00087C183EA9AE00E94EB14882309F046C01B
:107BF0008091A50A9091A60AAA27BB27888399831A
:107C0000AA83BB83E091AA0AF091AB0A80818D839D
:107C1000E091AA0AF091AB0A81818E83E091AA0AD1
:107C2000F091AB0A82818F83E091AA0AF091AB0AAE
:107C300083818887E091AA0AF091AB0A84818987C1
:107C4000E091AA0AF091AB0A85818A87E091AA0A9D
:107C5000F091AB0A86818B87E091AA0AF091AB0A7A
:107C600087818C878091A90A8C8383EA9AE00E949D
:107C7000D9138823D1F781E090E03AC18EEA9AE0E7
:107C80000E94EB14882309F046C08091B00A9091BD
:107C9000B10AAA27BB2788839983AA83BB83E09173
:107CA000B50AF091B60A80818D83E091B50AF09112
:107CB000B60A81818E83E091B50AF091B60A82817D
:107CC0008F83E091B50AF091B60A83818887E091AD
:107CD000B50AF091B60A84818987E091B50AF091DE
:107CE000B60A85818A87E091B50AF091B60A868145
:107CF0008B87E091B50AF091B60A87818C878091D5
:107D0000B40A8C838EEA9AE00E94D9138823D1F7B3
:107D100081E090E0EDC089EB9AE00E94EB148823AB
:107D200009F046C08091BB0A9091BC0AAA27BB27E4
:107D300088839983AA83BB83E091C00AF091C10A2A
:107D400080818D83E091C00AF091C10A81818E8388
:107D5000E091C00AF091C10A82818F83E091C00A4C
:107D6000F091C10A83818887E091C00AF091C10A2D
:107D700084818987E091C00AF091C10A85818A8750
:107D8000E091C00AF091C10A86818B87E091C00A18
:107D9000F091C10A87818C878091BF0A8C8389EB1F
:107DA0009AE00E94D9138823D1F781E090E0A0C027
:107DB00084EC9AE00E94EB14882309F046C080917D
:107DC000C60A9091C70AAA27BB2788839983AA83EA
:107DD000BB83E091CB0AF091CC0A80818D83E09146
:107DE000CB0AF091CC0A81818E83E091CB0AF0918D
:107DF000CC0A82818F83E091CB0AF091CC0A8381F7
:107E00008887E091CB0AF091CC0A84818987E09140
:107E1000CB0AF091CC0A85818A87E091CB0AF09158
:107E2000CC0A86818B87E091CB0AF091CC0A8781BE
:107E30008C878091CA0A8C8384EC9AE00E94D913C3
:107E40008823D1F781E090E053C08FEC9AE00E9444
:107E5000EB14882309F046C08091D10A9091D20A90
:107E6000AA27BB2788839983AA83BB83E091D60A7C
:107E7000F091D70A80818D83E091D60AF091D70ADC
:107E800081818E83E091D60AF091D70A82818F8317
:107E9000E091D60AF091D70A83818887E091D60ACB
:107EA000F091D70A84818987E091D60AF091D70AA8
:107EB00085818A87E091D60AF091D70A86818B87DF
:107EC000E091D60AF091D70A87818C878091D50AF4
:107ED0008C838FEC9AE00E94D9138823D1F781E03C
:107EE00090E006C0188219821A821B8280E090E01E
:107EF000DF91CF910895CF93DF93DC018091DA0A6F
:107F0000882339F48AED9AE090930B0B80930A0B47
:107F100021C08091E60A882339F486EE9AE0909396
:107F20000B0B80930A0B16C08091F20A882339F458
:107F300082EF9AE090930B0B80930A0B0BC0809119
:107F4000FE0A882309F072C08EEF9AE090930B0B23
:107F500080930A0BE0910A0BF0910B0B0084F185E2
:107F6000E02DED018D818083E0910A0BF0910B0BE8
:107F70000084F185E02D8E818183E0910A0BF091E0
:107F80000B0B0084F185E02D8F818283E0910A0B39
:107F9000F0910B0B0084F185E02D88858383E091BF
:107FA0000A0BF0910B0B0084F185E02D8985848309
:107FB000E0910A0BF0910B0B0084F185E02D8A858E
:107FC0008583E0910A0BF0910B0B0084F185E02D85
:107FD0008B858683E0910A0BF0910B0B0084F18571
:107FE000E02D8C858783E0910A0BF0910B0B8C813F
:107FF0008783E0910A0BF0910B0B8D919C919483F8
:108000008383E0910A0BF0910B0B1286E0910A0B2F
:10801000F0910B0B1182E0910A0BF0910B0B128285
:10802000E0910A0BF0910B0B81E08083DF91CF91FF
:1080300008958FEE99E00E946D3C882361F18FEEE8
:1080400099E00E9477118FEE99E00E946D3C8823A1
:1080500011F18FEE99E00E9477118FEE99E00E9466
:108060006D3C8823C1F08FEE99E00E9477118FEE6E
:1080700099E00E946D3C882371F08FEE99E00E9498
:1080800077118FEE99E00E946D3C882321F08FEEEE
:1080900099E00E9477110895FF920F931F93CF9359
:1080A000DF93CDB7DEB760970FB6F894DEBF0FBE93
:1080B000CDBF20E0822F99278C01045F144FF80177
:1080C00080818C7F8083F22EF394BE016F5F7F4F9F
:1080D0008F2D0E947A3288898170982F990F990F7D
:1080E000990FF80180818370892B80832F2D2B308D
:1080F00008F360960FB6F894DEBF0FBECDBFDF91D8
:10810000CF911F910F91FF900895FC0180818370A2
:108110009927009719F0019731F0089580818D72A9
:108120008162808308959081892F807FA1F493FDDF
:1081300005C0892F8E7F866080830895808182FFAD
:1081400003C08B7F808303C08081846080838081B3
:108150008C7F826080830895FC01808183709927E1
:1081600081309105BCF0833091051CF0039731F00C
:10817000089580818F708362808308959081892F14
:10818000807F41F4892F8C7F808393FD03C0892FEA
:10819000887F808308959927853C910509F457C00D
:1081A000863C9105ACF4823C9105C9F1833C910574
:1081B0003CF4803C910519F1813C910541F17AC074
:1081C000833C910509F45EC0843C9105C1F172C005
:1081D000813D910561F1823D910544F4863C910514
:1081E000F1F1873C910509F442C064C0823D9105DC
:1081F00009F450C0833D910509F454C05BC0309B25
:1082000003C081E090E0089580E090E00895319906
:1082100003C081E090E0089580E090E008953299F5
:1082200003C081E090E0089580E090E008954999CE
:1082300003C081E090E0089580E090E008953499D3
:1082400003C081E090E0089580E090E008953599C2
:1082500003C081E090E0089580E090E008953699B1
:1082600003C081E090E0089580E090E0089586B139
:10827000992787FD9095809590958827990F881F5D
:1082800099270895339903C081E090E0089580E034
:1082900090E008954A9903C081E090E0089580E05D
:1082A00090E008954B9903C081E090E0089580E04C
:1082B00090E0089580E090E0089530E0832F9927C2
:1082C000FC01E45FF44F2081822F807F41F0822FF8
:1082D000807F982F9051822F8F70892B80833F5FF2
:1082E0003B3060F3ECE0FBE0309B04C0CF010E9428
:1082F000854003C0CF010E94AC40EDE0FBE0319926
:1083000004C0CF010E94854003C0CF010E94AC4051
:10831000EEE0FBE0329904C0CF010E94854003C02B
:10832000CF010E94AC40EFE0FBE0499904C0CF01CF
:108330000E94854003C0CF010E94AC40E0E1FBE019
:10834000349904C0CF010E94854003C0CF010E9430
:10835000AC40E1E1FBE0359904C0CF010E948540CB
:1083600003C0CF010E94AC40E2E1FBE0369904C0BB
:10837000CF010E94854003C0CF010E94AC40E3E1E1
:10838000FBE0379904C0CF010E94854003C0CF01B4
:108390000E94AC40E4E1FBE0339904C0CF010E94AD
:1083A000854003C0CF010E94AC40E5E1FBE04A9963
:1083B00004C0CF010E94854003C0CF010E94AC40A1
:1083C000E6E1FBE04B9904C0CF010E94854008958F
:1083D000CF010E94AC4008959927853C910509F48E
:1083E00051C0863C9105ACF4823C9105B1F1833CCF
:1083F00091053CF4803C910511F1813C910531F1EE
:108400006BC0833C910509F452C0843C910599F1FD
:1084100063C0813D910541F1823D91053CF4863C6C
:108420009105B9F1873C9105D9F156C0823D91057E
:1084300009F444C0833D910509F447C04DC08091C3
:108440000C0B8695869581709927089580910D0B68
:108450008695869581709927089580910E0B869553
:10846000869581709927089580910F0B8695869542
:108470008170992708958091100B8695869581705B
:10848000992708958091110B86958695817099277B
:1084900008958091120B869586958170992708958D
:1084A0008091130B86958695817099270895809108
:1084B000140B869586958170992708958091150BE8
:1084C000869586958170992708958091160B8695DB
:1084D00086958170992708958EEF90E00895109207
:1084E000B60087E08093B0001092B2008EE48093D3
:1084F000B30082E08093700008950E946F42109252
:10850000190B10921A0B10921B0B10921C0B10924D
:10851000210B1092220B0E944C400E94FE050E94EB
:10852000012E0895CF93C82F8091170B882311F047
:108530001092170BA8950E941940C23011F00E94AA
:10854000EC3BC23009F46FC08091180B882309F40A
:1085500044C08091180B81508093180B8091190BA7
:108560008F5F8093190B823040F01092190B0E949C
:108570005D410E94BF150E94380780911A0B8F5FE2
:1085800080931A0B843040F010921A0B0E943D1613
:108590000E94F5530E94005180911B0B8F5F8093C6
:1085A0001B0B8A3030F010921B0BC13011F00E946F
:1085B0005F1180911C0B8F5F80931C0B843168F0DE
:1085C00010921C0B8091210B8F5F8093210B0E94D6
:1085D00085360E9465170E9414118091210B8A3004
:1085E00010F11092210B80911D0B90911E0BA09108
:1085F0001F0BB091200B0196A11DB11D80931D0B87
:1086000090931E0BA0931F0BB093200B0E94092F79
:108610008091220B8F5F8093220B8C3320F010927D
:10862000220B0E94C82ECF91089580911D0B90912E
:108630001E0BA0911F0BB091200BBC01CD01089522
:108640001F920F920FB60F9211248F931092B200C7
:1086500081E08093170B8091180B8F5F8093180B2C
:108660008F910F900FBE0F901F9018950E949F4FF3
:108670000E94525160E076E980E090E00E946D51E6
:10868000089504C00E94E54F0E9438500E94CF4FC9
:108690008823C1F70895FC0190E061506F3F21F0FD
:1086A000819198276150E0F7892F992708950F93BA
:1086B0001F938C01FC0181818150682FC8010196B4
:1086C0000E944B43F801808381819927BC01C80136
:1086D0000E9400501F910F910895AF92BF92CF92C8
:1086E000DF92EF92FF920F931F93CF93DF93CDB75B
:1086F000DEB7C35ED0400FB6F894DEBF0FBECDBF6D
:108700006C01FC0181818150682FC60101960E9495
:108710004B43D6019C91981711F00C942D4FF60104
:108720008281882309F0F8C08381992781359105DA
:1087300009F449C0823591053CF48033910589F0F4
:108740008035910561F1E8C08335910509F48EC04B
:10875000833591050CF478C08435910509F4B2C0D5
:10876000DBC08E01035D1F4F80E5D8011D928A9505
:10877000E9F785E18EA71FA680E888ABF601848122
:1087800089AB992796012B5F3F4FAC01B901CE0110
:10879000C2960E94DB62C8010E945743BDC08E0191
:1087A000035D1F4F80E5D8011D928A95E9F785E0AA
:1087B0008EA71FA680EA88AB0E948F2C89ABC801C8
:1087C0000E945743A9C0F601B4800F2EFDE2EF2EA0
:1087D000FF24F02DEC0EFD1E80E5D7011D928A9539
:1087E000E9F789E18EA71FA681EA88AB8E010358BD
:1087F0001F4FB8018B2D0E94B92CB9AA8CE0FE0145
:10880000F296D8010D9001928A95E1F7F8018485DE
:1088100095859FAF8EAF8685FE01E05CFF4F80831C
:10882000F8018785FE01EF5BFF4F80839927AC013C
:10883000BE0163577F4FCE018E5B9F4F0E94DB626C
:10884000C7010E94574368C00E94472CFE01BD9695
:1088500080E5DF011D928A95E9F784E08EA71FA6C7
:1088600082EA88ABCF010E94574356C0F60145818A
:1088700056818481FE01ED51FF4F8083813108F0E4
:108880004BC080E5FE01BD9611928A95E9F787E11C
:108890008EA71FA683EA88AB5BAB4AABFE01ED5106
:1088A000FF4F808189ABFE01F4969927DA01019789
:1088B00024F00E94BF630192FACFCE018D960E94F0
:1088C00057432AC0F601458156818481FE01ED514E
:1088D000FF4F8083813100F5F60137969927DA0141
:1088E000019724F001900E94CC63FACFDE019D969F
:1088F00080E5FD0111928A95E9F787E08EA71FA612
:1089000084EA88AB5BAB4AABFE01ED51FF4F80813F
:1089100089ABCD010E945743F6018281813011F06D
:108920000C94364F83819927AA27BB27FC013197E6
:10893000EB36F10510F00C941F4FE65BFF4FEE0F86
:10894000FF1F0590F491E02D09940E949F2AF601E3
:10895000B4808B2D8150823210F00C94364F20E081
:10896000AE01475F5F4F822F9927DA01A80FB91F29
:10897000F601E80FF91F82858C932F5F2F3098F353
:10898000F6018581898386818A8387818B83838DA4
:10899000948D9E838D83858D8F8380858887818547
:1089A0008C83818D888F828D898F6B2DCE0101966E
:1089B0000E94C6316B2DCE0101960E94621F1DA63A
:1089C00085E08EA711E01FA781E888AB19AACE0128
:1089D0008D960E945743812F0E9492420C94364FED
:1089E000F601B4808B2D8150823208F047C06B2D88
:1089F000CE0101960E940B328EE18EA781E08FA7F7
:108A000082E888ABB9AA89818AAB8A818BAB8B81DA
:108A10008CAB8C818EAB8D819E81FE01E85BFF4F1C
:108A2000918380838F81FE01E65BFF4F808320E08E
:108A3000BE016F5F7F4FAE01475F5F4F822F992767
:108A4000DC01A60FB71FFA01E80FF91F8081FD01B5
:108A500086AB2F5F2F3090F388858DAB888DFE011C
:108A6000EA5BFF4F8083898DFE01E95BFF4F8083C6
:108A7000CE018D960E9457430C94364FFFEFBF16E0
:108A800011F00C94364FFE01ED51FF4F1082FE01A4
:108A9000ED51FF4F8081982F823210F00C94364FA9
:108AA0000F2EF3EEEF2EFF24F02DEC0EFD1E6E01C7
:108AB0000894C11CD11C8E01075F1F4F892F8F5F47
:108AC000682FCE0101960E940B328EE18EA781E0C5
:108AD0008FA782E888ABD7018C918F5F89AB8981A2
:108AE0008AAB8A818BAB8B818CAB8C818EAB8D8179
:108AF0009E81FE01E85BFF4F918380838F81FE01A1
:108B0000E65BFF4F808320E0822F9927DC01AC0DCC
:108B1000BD1DF801E80FF91F8081FD0186AB2F5FB5
:108B20002F3090F388858DAB888DFE01EA5BFF4F77
:108B30008083898DFE01E95BFF4F8083CE018D9696
:108B40000E94574381E00E949242D7018C918F5F2F
:108B50008C93982F823208F4B1CF0C94364F0E9438
:108B60009F2AF601B480AE0143585F4F96012B5FF8
:108B70003F4F8FE0DA01F90101900D928A95E1F7FC
:108B8000F6018489FA018787BA018B2D0E945D3234
:108B900081E08FA783E888ABB9AA85E08EA7CE01D4
:108BA0008D960E9457430C94364FF601B4808B2D5E
:108BB00081508A3010F581E08FA784E888ABB9AA8C
:108BC0008E0103581F4FB8018B2D0E947A328FE01F
:108BD000FE01F296D8010D9001928A95E1F7F80115
:108BE0008785FE01EF5BFF4F808385E18EA7CE0175
:108BF0008D960E9457430C94364FFFEFBF1611F02D
:108C00000C94364FFE01ED51FF4F1082FE01ED51E5
:108C1000FF4F8081982F8B3010F00C94364FBB247F
:108C2000B3948E0103581F4F0F2EFFE0AF2EF02D8F
:108C30000F2EF1E4EF2EFF24F02DEC0EFD1E0F2E73
:108C4000F3EECF2EDD24F02DCC0EDD1EBFA684E882
:108C500088AB892F8F5F89ABB8010E947A32FE0101
:108C6000F296D8012A2D0D9001922A95E1F7F8018C
:108C70008785D7018C9385E18EA7CE018D960E94C2
:108C800057438B2D0E949242F60180818F5F808333
:108C9000982F8B30D8F20C94364F0E949F2A0E9456
:108CA000FA19A8950E94081DA8950E94701EA89503
:108CB0000E947A10A8950E94C153A8950E9455065B
:108CC000A8950E946E2E0E94F90E81E08FA786E87B
:108CD00088AB84E08EA7CE018D960E9457430C94FA
:108CE000364F84E18EA781E08FA787E888AB8DE0BF
:108CF000A8E7B1E0FE01F1960D9001928A95E1F7A7
:108D00000E9415439B01AC01AA27BB278EAFBB274E
:108D1000A52F942F832F8FAFFE01E05CFF4F2083A0
:108D2000CE018D960E9457430C94364F0C94000050
:108D30000C94364FC60104960E94543081E08FA7F0
:108D400089E888AB84E08EA7CE018D960E945743B8
:108D50000C94364F81E08FA78AE888AB8CE08EA711
:108D6000CE01C1960E946430CE018D960E94574379
:108D70000C94364FCE0187960E94EB2781E08FA797
:108D800081EA88AB8FA189AB88A58AAB89A58BAB1B
:108D90008AA58CAB8BA58DAB8CA58EAB8AE08EA7FC
:108DA000CE018D960E9457430C94364FF601B48045
:108DB000F1E2FB1500F1BE016E5D7F4F8B2D0E942D
:108DC000DD2881E08FA782EA88ABB9AA8BA18BABA3
:108DD0008CA18EAB8AA18AAB8DA19EA1892F9927E8
:108DE0008CAB8DA18DAB8AE08EA7CE018D960E94B3
:108DF00057430C94364F2FEFB21611F00C94364FA8
:108E0000FE01ED51FF4F1082FE01ED51FF4F8081B9
:108E1000982F823210F00C94364FFF24F3948F0178
:108E2000BE016E5D7F4F892F8F5F0E94DD28FFA6F8
:108E300082EA88ABD8018C918F5F89AB8BA18BAB19
:108E40008CA18EAB8AA18AAB8DA19EA1892F992777
:108E50008CAB8DA18DAB8AE08EA7CE018D960E9442
:108E600057438F2D0E949242F80180818F5F80834B
:108E7000982F8232A8F20C94364FCE014A960E9467
:108E8000A7298AE08EA781E08FA780EA88AB88A116
:108E900089AB8E8D8AAB8A8D9B8D892F99278BAB61
:108EA0008A8D8CAB8D8D8DAB8C8D8EABCE018D96DE
:108EB0000E945743DBC7F601648180E00E941E22B6
:108EC00084E08EA781E08FA783EA88ABCE018D96E0
:108ED0000E945743CBC7DE01A353BF4FF6018481E5
:108EE0008C938581FD018183F6018681FD0182835A
:108EF000F6018781FD018383F6018085FD0184836E
:108F0000F6018185FD018583F6018285FD01868359
:108F1000F6018385FD018783CD010E94262284E02E
:108F20008EA781E08FA784EA88ABCE018D960E9440
:108F300057439CC7FE01E358FF4FA0E0B0E080E13B
:108F400090E021E08030920719F40E94C76303C0CB
:108F5000182E0E94C763F60184819581A681B7818E
:108F6000FE01EF57FF4F80839183A283B383DE011D
:108F7000A358BF4FF6018085FD018087F6018185EA
:108F8000FD018187F6018285FD018287A0E0B0E0C6
:108F900080E190E021E08030920719F40E94D863CC
:108FA00003C0182E0E94D86384E08EA781E08FA7AB
:108FB00080EC88ABCE018D960E94574357C7FE01C7
:108FC000E358FF4FA0E0B0E080E190E021E0803086
:108FD000920719F40E94C76303C0182E0E94C7634A
:108FE0008BE08EA781E08FA781EC88ABFE01EF5765
:108FF000FF4F80819181A281B38189AB9AABABABEA
:10900000BCABFE01E358FF4F80858DAB81858EABF5
:1090100082858FABCE018D960E94574327C78AE386
:109020008EA781E08FA780ED88ABFE01F196A8E8BE
:10903000B0E082E190E021E08030920719F40E94D4
:10904000C76303C0182E0E94C763FE01ED5BFF4F8C
:10905000AAE9B0E082E190E021E08030920719F4C3
:109060000E94C76303C0182E0E94C763FE01EB5A1B
:10907000FF4FADEBB0E082E190E021E0803092075D
:1090800019F40E94C76303C0182E0E94C763CE0163
:109090008D960E945743EAC684E18EA781E08FA790
:1090A0008EED88ABFE01F196ACEAB0E080E190E095
:1090B00021E08030920719F40E94C76303C0182E84
:1090C0000E94C763CE018D960E945743CFC60E946F
:1090D0006E2E84E08EA781E08FA781ED88ABCE0154
:1090E0008D960E945743C2C688E08EA781E08FA765
:1090F0008FED88AB0E94002F8BAB0E94042F9AABA0
:1091000089ABFE01ED51FF4FACEBB0E081E090E0A8
:1091100021E08030920719F40E94C76303C0182E23
:109120000E94C763FE01ED51FF4F80818CABCE01E1
:109130008D960E9457439AC6FE01E358FF4F80E583
:10914000DF011D928A95E9F7ACEBB0E081E090E099
:1091500021E08030920719F40E94D86303C0182ED2
:109160000E94D863FE01E358FF4FA5E8B0E081E01C
:1091700090E021E08030920719F40E94D86303C088
:10918000182E0E94D863FE01E358FF4FA6E8B0E016
:1091900082E090E021E08030920719F40E94D863C9
:1091A00003C0182E0E94D86384E08EA781E08FA7A9
:1091B00080EE88ABCE018D960E94574357C6F601CC
:1091C0008581968190936D0E80936C0E878190853A
:1091D00090936F0E80936E0E818592859093710EA1
:1091E0008093700E83858093720E84858093730EB6
:1091F00085858093740E878590899093770E8093F0
:10920000760E86858093750EECE6FEE0A0E7B0E072
:109210008CE090E021E08030920719F40E94D8633E
:1092200003C0182E0E94D86385E08EA791E09FA707
:1092300085EA88AB99ABCE018D960E94574316C63E
:1092400081E18EA781E08FA786EA88AB19AA809179
:10925000E200863269F48091E300843049F4809121
:10926000E400833129F484E690E09BAB8AAB46C0EE
:109270008091E2008E3169F48091E300843049F4FA
:109280008091E400833129F48DE790E09BAB8AABB9
:1092900035C08091E2008E3069F48091E300843023
:1092A00049F48091E400833129F48AEF90E09BAB8C
:1092B0008AAB24C08091E200863069F48091E3009B
:1092C000843049F48091E400833129F484EF91E003
:1092D0009BAB8AAB13C08091E200823069F480912D
:1092E000E300843049F48091E400833129F488EE6E
:1092F00093E09BAB8AAB02C01BAA1AAA80916E0EA8
:1093000090916F0E9DAB8CAB8091700E9091710E11
:109310009FAB8EAB8091720E88AF8091730E89AF38
:109320008091740E8AAF8091760E9091770E9DAFEA
:109330008CAF8091750E8BAFCE018D960E945743F6
:1093400095C5DE01AB52BF4FF60184818C938581B8
:10935000FD018183D60116968CE0FE01E952FF4F94
:109360000D9001928A95E1F7FE01ED51FF4F1082B9
:10937000FE01ED51FF4F8081982F8C30A0F49E01AB
:109380002B523F4FDF01F901E90FF11D8281882344
:1093900021F08F3F11F0815082838C918F5F8C93ED
:1093A000982F8C3080F3CE018B529F4F0E94063055
:1093B00084E08EA781E08FA787EA88ABCE018D96E7
:1093C0000E94574353C58E010B521F4FC8010E9484
:1093D000243082E18EA781E08FA788EA88ABD8018C
:1093E0008C9189ABF80181818AABFE01ED51FF4F71
:1093F0001082FE01ED51FF4F8081982F8C3080F458
:109400009801DF01F901E90FF11D82818F3F11F011
:109410008F5F82838C918F5F8C93982F8C3090F329
:109420008CE0DE01A952BF4FFE01F3960D90019230
:109430008A95E1F7CE018D960E94574317C5F60134
:109440008481FE01E358FF4F8083D60115968EE09C
:10945000FE01E258FF4F0D9001928A95E1F7FE015F
:10946000ED51FF4F1082FE01ED51FF4F8081982F8B
:109470008E30A0F49E0123583F4FDF01F901E90F20
:10948000F11D8181882321F08F3F11F0815081836C
:109490008C918F5F8C93982F8E3080F3DE01A358D0
:1094A000BF4FF6018389FD018787F6018489FD019D
:1094B000808BD60155968EE0FE01E257FF4F0D904E
:1094C00001928A95E1F7FE01ED51FF4F1082FE01F6
:1094D000ED51FF4F8081982F8E30A0F49E012358CC
:1094E0003F4FDF01F901E90FF11D8189882321F048
:1094F0008F3F11F08150818B8C918F5F8C93982FCF
:109500008E3080F3CE0183589F4F0E94343084E028
:109510008EA781E08FA789EA88ABCE018D960E9445
:109520005743A4C48E0103581F4FC8010E94443002
:1095300083E28EA781E08FA78AEA88ABD8018C915D
:1095400089ABFE01ED51FF4F1082FE01ED51FF4F3F
:109550008081982F8E3080F49801DF01F901E90FA6
:10956000F11D81818F3F11F08F5F81838C918F5F1F
:109570008C93982F8E3090F38EE0DE01A258BF4F6F
:10958000FE01F2960D9001928A95E1F7DE01A35853
:10959000BF4FFD018785FE01E05CFF4F8083FD0129
:1095A0008089FE01EF5BFF4F8083FE01ED51FF4F8D
:1095B0001082FE01ED51FF4F8081982F8E3080F494
:1095C0009D01DF01F901E90FF11D81898F3F11F044
:1095D0008F5F818B8C918F5F8C93982F8E3090F35F
:1095E0008EE0DE01A257BF4FFE01EE5BFF4F0D90F4
:1095F00001928A95E1F7CE018D960E94574336C4B9
:10960000F601B48085819927982F88272681820FBB
:10961000911DBC018B2D0E94222A85E08EA781E03E
:109620008FA782EC88ABB9AACE018D960E945743D2
:109630001DC4F601B4808CE08EA781E08FA783EC77
:1096400088ABB9AA8B2D0E94E0298AAB8B2D0E9492
:10965000FC29892F99278BAB8B2D0E94FC298CAB81
:109660008B2D0E944B2A892F99278DAB8B2D0E9421
:109670004B2A8EAB8B2D0E94632A892F99278FABA3
:109680008B2D0E94632A88AFCE018D960E9457438E
:10969000EDC320E0F601848181FD21E0F6018481A3
:1096A00082FD2260F6018181863029F46581822F56
:1096B0000E947B2ADBC360E0822F0E947B2AD6C3F4
:1096C0000E94802A84E08EA781E08FA785EC88AB7A
:1096D000CE018D960E945743C9C3F601B4809E0106
:1096E00023583F4F9581492F4170D9018C91887F34
:1096F0009670842B892B8C9386819781F9019283B4
:109700008183F60180859185F90194838383F60135
:109710008685F9018187F6018785F9018287F6013F
:1097200082859385F90196838583F60184859585E5
:10973000F90190878783F6018089F9018387F60113
:109740008189F9018487F6018289F9018587F6010B
:109750008389F9018687D60154968FE0FE01E4578C
:10976000FF4F0D9001928A95E1F7F60183A1F9016F
:10977000868FF60184A1F901878FF60185A1F90191
:1097800080A3F60186A1F90181A315E0D601979681
:10979000FE01E156FF4F812F0D9001928A95E1F76E
:1097A000F60184A595A5A6A5B7A5F90187A390A75D
:1097B000A1A7B2A7F60180A9F90183A7B9018B2D52
:1097C0000E94E63081E08FA782ED88AB1EA7B9AA80
:1097D000CE018D960E94574349C3F601B4808E0195
:1097E00003581F4FB8018B2D0E941E3181E08FA7B7
:1097F00083ED88AB81E38EA7B9AAD8019C91292F6C
:1098000021708AA9887F9670822B892B8AABF801F8
:10981000818192819CAB8BAB838194819EAB8DAB1C
:1098200081858BAF82858CAF8581968198AF8FAB18
:10983000878190859AAF89AF83858DAF84858EAF00
:1098400085858FAF8685FE01E05CFF4F80838FE0CA
:10985000DE01A457BF4FFE01EF5BFF4F0D90019259
:109860008A95E1F7F801868DFE01E05BFF4F80836A
:10987000F801878DFE01EF5AFF4F8083F80180A128
:10988000FE01EE5AFF4F8083F80181A1FE01ED5ADF
:10989000FF4F808385E0DE01A156BF4FFE01EC5AE9
:1098A000FF4F0D9001928A95E1F7F80187A190A5ED
:1098B000A1A5B2A5FE01E75AFF4F80839183A28341
:1098C000B383F80183A5FE01E35AFF4F8083CE01E5
:1098D0008D960E945743CAC2F601B480AE01435828
:1098E0005F4F828DDA018C93838DFA018183F601BB
:1098F000848DFA018283F6018681FA018383F60161
:109900008781FA018483F6018085FA018583F60157
:109910008185FA018683F6018285FA018783F60143
:10992000858DFA01878BC6010B962FE0FE01EB5760
:10993000FF4FDC010D9001922A95E1F7BA018B2DC2
:109940000E94563181E08FA784ED88AB85E08EA719
:10995000B9AACE018D960E94574388C2F601B48001
:109960008E0103581F4FB8018B2D0E948E3181E06C
:109970008FA785ED88AB8FE18EA7B9AAD8018C910E
:10998000FE01E95BFF4F8083F8018181FE01E85B06
:10999000FF4F8083F8018281FE01E75BFF4F8083E8
:1099A000F80183818BAB84818CAB85818DAB868103
:1099B0008EAB87818FAB8789FE01E65BFF4F80838B
:1099C0008FE0DE01AB57BF4FFE01F8960D9001927C
:1099D0008A95E1F7CE018D960E94574347C2F60162
:1099E0003496AAEEB8E082E090E021E08030920761
:1099F00019F40E94D86303C0182E0E94D86381E036
:109A00008FA783EE88AB84E08EA7CE018D960E944F
:109A100057432CC281E08FA784EE88AB84E18EA7E8
:109A2000FE01F196AAEEB8E082E090E021E08030FD
:109A3000920719F40E94C76303C0182E0E94C763DF
:109A4000CE018D960E94574311C2F601B480C60123
:109A50000596BC018B2D0E94743081E08FA788EDA4
:109A600088AB85E08EA7B9AACE018D960E94574398
:109A7000FDC1F601B48081E08FA789ED88AB8EE14E
:109A80008EA7B9AABE016E5C7F4F8B2D0E94AD30B0
:109A9000CE018D960E945743E9C1F60184818093DF
:109AA000790E858180937A0E868180937B0E8781E3
:109AB00080937C0E808580937D0E818580937E0EC1
:109AC000828580937F0E83858093800EE9E7FEE098
:109AD000AEE6BFE088E090E021E08030920719F424
:109AE0000E94D86303C0182E0E94D86381E08FA71C
:109AF00085EE88AB84E08EA7CE018D960E945743F9
:109B0000B5C181E08FA786EE88AB8CE08EA78091EF
:109B1000790E89AB80917A0E8AAB80917B0E8BABEC
:109B200080917C0E8CAB80917D0E8DAB80917E0EF2
:109B30008EAB80917F0E8FAB8091800E88AFCE016F
:109B40008D960E94574392C1F6013496AEE8BFE06D
:109B50008CE490E021E08030920719F40E94D863F1
:109B600003C0182E0E94D863F60184818093810E71
:109B70008581982F97708091820E887F892B8093A2
:109B8000820E87898093830E808D982F97708091A5
:109B9000840E887F892B8093840E82A58093850E06
:109BA00083A5982F97708091860E887F892B80934C
:109BB000860E85AD8093870E86AD982F9770809125
:109BC000880E887F892B8093880E81E08FA787EE8F
:109BD00088AB84E08EA7CE018D960E94574346C184
:109BE00081E08FA788EE88AB80E58EA7FE01F19615
:109BF000AEE8BFE08CE490E021E08030920719F4F9
:109C00000E94C76303C0182E0E94C763CE018D96C1
:109C10000E9457432BC1F6013496AAEDBFE089E0BC
:109C200090E021E08030920719F40E94D86303C0CD
:109C3000182E0E94D863F6013D96A3EEBFE089E09E
:109C400090E021E08030920719F40E94D86303C0AD
:109C5000182E0E94D86381E08FA789EE88AB84E03C
:109C60008EA7CE018D960E94574300C181E08FA739
:109C70008AEE88AB87E18EA7FE01F196AAEDBFE0E0
:109C800089E090E021E08030920719F40E94C763D8
:109C900003C0182E0E94C763FE01FA96A3EEBFE030
:109CA00089E090E021E08030920719F40E94C763B8
:109CB00003C0182E0E94C763CE018D960E945743A1
:109CC000D5C0C60105960E94E83281E08FA786EDD7
:109CD00088AB85E08EA7CE018D960E945743C6C003
:109CE00081E08FA787ED88AB8DE18EA7CE01C2966C
:109CF0000E94F832CE018D960E945743B7C0F601FC
:109D0000B480C60104960E94083381E08FA78AEDD3
:109D100088AB85E08EA7B9AACE018D960E945743E5
:109D2000A5C0F601B48081E08FA78BED88AB8AE4F3
:109D30008EA7BE016F5C7F4F8B2D0E943533CE0105
:109D40008D960E94574392C0F601B4808B2D0E94DD
:109D5000E31081E08FA78CED88ABB9AA85E08EA7D0
:109D6000CE018D960E94574381C0F60144815581F2
:109D700081E08FA78DED88AB86E18EA75AAB49AB0A
:109D8000FE01ED51FF4F1082FE01ED51FF4F80812A
:109D9000982F8031C8F48E010F5F1F4FBF01892FAC
:109DA00099279C01200F311F840F951FAA27BB27DD
:109DB000ABBFFC018791F90182ABDB018C918F5F16
:109DC0008C93982F803158F3CE018D960E94574383
:109DD0004DC0F6013496AEE5BFE080E190E021E0B1
:109DE0008030920719F40E94D86303C0182E0E9495
:109DF000D86381E08FA781EE88AB84E08EA7CE0187
:109E00008D960E94574332C081E08FA782EE88ABC7
:109E100084E18EA7FE01F196AEE5BFE080E190E01F
:109E200021E08030920719F40E94C76303C0182E06
:109E30000E94C763CE018D960E94574317C081E0F0
:109E40008FA780E888AB85E08EA7F601838189AB78
:109E5000CE018D960E94574309C085E08EA71FA6AC
:109E600081E088ABCE018D960E945743CD51DF4FE4
:109E70000FB6F894DEBF0FBECDBFDF91CF911F911B
:109E80000F91FF90EF90DF90CF90BF90AF9008952B
:109E9000CF93DF93CDB7DEB72A970FB6F894DEBF26
:109EA0000FBECDBF81E08B8388E88C8384E08A83FA
:109EB000CE0101960E9457432A960FB6F894DEBF52
:109EC0000FBECDBFDF91CF9108950F931F93CF9316
:109ED000DF93CDB7DEB7C055D0400FB6F894DEBFE4
:109EE0000FBECDBF8A0121E02B832DE52C839E83FD
:109EF0008D836F8320E0261780F4AE01485F5F4FAB
:109F0000822F9927DA01A80FB91FF801E80FF91F6E
:109F100080818C932F5F261798F38FE08A83CE0180
:109F200001960E945743C05BDF4F0FB6F894DEBF27
:109F30000FBECDBFDF91CF911F910F91089548ECD7
:109F400050E060E070E084E29BE00E94E8621092E2
:109F5000EC0B1092ED0B1092230B0895382F2091EB
:109F6000ED0B84E29BE0FC01E20FF11D3083809158
:109F7000ED0B8F5F8093ED0B8091230B8F5F8093B0
:109F8000230B8091230B883C18F00E949F4F08956B
:109F90008091ED0B883C10F01092ED0B089590919C
:109FA000ED0B8091EC0B981738F08091ED0B9091B0
:109FB000EC0B891B992708959091ED0B8091EC0B88
:109FC000981B892F8853992708952091EC0B84E2E0
:109FD0009BE0FC01E20FF11DE0818091EC0B8F5FB3
:109FE0008093EC0B8091230B81508093230B809105
:109FF000EC0B883C10F01092EC0B8E2F99270895F3
:10A000000F931F93CF93DF93EC018B0180EC0E94A1
:10A010009351015010408FEF0F3F180709F18881CD
:10A020009927803C910521F08B3D910541F00EC0B0
:10A030008BED0E9493518CED0E9493510AC08BEDE1
:10A040000E9493518DED0E94935103C088810E941C
:10A0500093512196015010408FEF0F3F1807F9F6EA
:10A0600080EC0E949351DF91CF911F910F91089541
:10A070000F931F93382F8091EE0B9927009719F0BB
:10A080000197C1F059C0303C09F056C01092EF0B57
:10A090002091EF0B81EF9BE0FC01E20FF11D30837B
:10A0A0002F5F2093EF0B81E08093EE0B84E680938B
:10A0B000F00B42C0303C99F58091EF0B8230F0F00C
:10A0C0008091EF0B01EF1BE0F801E80FF11D3083E9
:10A0D0008F5F8093EF0B82E08093EE0B1092F00B7A
:10A0E000A8016091EF0BC8010E94A750C8010E940F
:10A0F0006D431092EE0B1092EF0B1EC01092EF0BFF
:10A100002091EF0B81EF9BE0FC01E20FF11D30830A
:10A110002F5F2093EF0B84E68093F00B0DC020910E
:10A12000EF0B81EF9BE0FC01E20FF11D308380918A
:10A13000EF0B8F5F8093EF0B8091EF0B893620F050
:10A140001092EE0B1092EF0B1F910F910895FC01EE
:10A15000DA0161506F3FF1F02081822F9927803C16
:10A16000910521F08B3D910519F010C0319610C07A
:10A1700031962081822F99278C3D910521F08D3DCC
:10A18000910519F003C020EC01C02BED2D93319601
:10A19000615010F708958091F00B882389F0809129
:10A1A000F00B81508093F00B9091F00B992341F4C8
:10A1B0008091EE0B813021F49093EF0B9093EE0B96
:10A1C000089585B1807F85B984B1876084B981E5C0
:10A1D0008CBD81E08DBD08958EBD0DB407FEFDCF11
:10A1E0008EB5992708950E9450519C9AA4988FE0AB
:10A1F00080935B0CA4986A9862980895A498089537
:10A20000CF93DF93CDB7DEB728970FB6F894DEBFB4
:10A210000FBECDBFA49B18C0629914C080915A0C88
:10A22000853050F0A4980E941F2082E28093120192
:10A230001092890E1092780E80915A0C8F5F809345
:10A240005A0C02C010925A0CCE0101960E94A72906
:10A2500029813A8181E590E0289FA001299F500D36
:10A26000389F500D1124CA01880F892F881F990B20
:10A2700091950E9451518D81882319F48F818823F3
:10A2800011F0A49A01C0A49828960FB6F894DEBFE6
:10A290000FBECDBFDF91CF91089580935B0C0895E1
:10A2A0000895089510925D0C10925C0C86E08093E6
:10A2B000C20088E98093C10060E875E280E090E028
:10A2C0000E946D5181E08093F20E1092F30E08957A
:10A2D00090935D0C80935C0C08959B01AC01DC01B4
:10A2E000CB01689412F8880F991FAA1FBB1F169400
:10A2F000D1F780509C4DAB40BF4F689413F8220FAC
:10A30000331F441F551F1694D1F7BC01CD010E9485
:10A310004B63DA01C9010197292F33272093C50028
:10A320008093C4000895982F8091C00085FFFCCFD2
:10A330009093C60008950F931F93CF93DF938C01E2
:10A34000EB0121978FEFCF3FD80751F0F8018191B2
:10A350008F010E9493512197FFEFCF3FDF07B1F7A5
:10A3600081E090E0DF91CF911F910F9108951F92AE
:10A370000F920FB60F9211242F933F934F935F9339
:10A380006F937F938F939F93AF93BF93EF93FF93BD
:10A390008091C6000E94AE4FFF91EF91BF91AF91A7
:10A3A0009F918F917F916F915F914F913F912F91ED
:10A3B0000F900FBE0F901F901895DC01FB014150CC
:10A3C00050408FEF4F3F580741F081918D9341509E
:10A3D00050408FEF4F3F5807C1F70895DC01FB0154
:10A3E000415050408FEF4F3F580769F091918D9148
:10A3F000891719F081E090E00895415050408FEFA7
:10A400004F3F580799F780E090E00895CF93DF938E
:10A41000DC01FB0160E0462F91E0562F8081803205
:10A4200031F4692F9F5F319680818032D1F3808132
:10A43000882379F08081803219F4442309F4492F6C
:10A440008081803209F040E09F5F319680818823CF
:10A4500089F7442331F48081882311F4492F01C006
:10A46000462F262F3327E901C91BD109EC0FFD1F09
:10A470003196842F9927821B930B01971816190682
:10A4800024F4942F961B915001C090E091509F3F6F
:10A4900029F081918D935F5F9150D8F71C925F5F97
:10A4A000852F9927DF91CF910895FC0190E081914C
:10A4B000882331F09F5F8191882311F09F3FD1F76E
:10A4C000892F99270895DC01FB018081882329F0D9
:10A4D00081918D9380818823D9F71C9208950F93E1
:10A4E0001F93CF93DF93082F162FFA0141E0C0E1AD
:10A4F000D7E2C901BE010E9438636115710581F080
:10A500006C9FC0016D9F900D7C9F900D1124281BA6
:10A51000390B862F805D8193440F01E015E00AC05E
:10A52000153040F0002319F080E3819302C080E2EF
:10A5300081934F5FC8EED3E0C901BE010E9438632A
:10A540006115710581F06C9FC0016D9F900D7C9F1E
:10A55000900D1124281B390B862F805D81934F5F4E
:10A5600001E014E00AC0143040F0002319F080E349
:10A57000819302C080E281934F5FC4E6D0E0C901BD
:10A58000BE010E9438636115710581F04F5F6C9FB9
:10A59000C0016D9F900D7C9F900D1124281B390BDD
:10A5A000862F805D819301E013E00AC0133040F0F4
:10A5B0004F5F002319F080E3819302C080E2819312
:10A5C000C9016AE070E00E9438636115710591F07D
:10A5D0004F5FCB01880F991F880F991F880F991F14
:10A5E000860F971F860F971F281B390B862F805DBC
:10A5F00081930AC0123040F04F5F002319F080E3CE
:10A60000819302C080E28193822F805D81931082CA
:10A61000842F9927DF91CF911F910F910895FC010D
:10A62000262F862F82958F708A3038F06AE00E943C
:10A630001863892F8F5B819309C0862F82958F7055
:10A640006AE00E941863892F805D8193822F8F704A
:10A650008A3038F06AE00E941863892F8F5B80830C
:10A660000895822F8F706AE00E941863892F805DA1
:10A6700080830895EF92FF920F931F937C018B01CB
:10A68000872F9927682FC7010E940F53C801907028
:10A69000682FC7010E940F531F910F91FF90EF90F9
:10A6A0000895CF92DF92EF92FF920F931F936C0168
:10A6B0007A018B01CB01AA27BB27BC01C6010E94EE
:10A6C0003A53D801C701A070B070BC01C6010E9406
:10A6D0003A531F910F91FF90EF90DF90CF90089524
:10A6E0001F93CF93DF93CDB7DEB768970FB6F8947B
:10A6F000DEBF0FBECDBF10E0BE016F5F7F4F812F69
:10A700000E948E31412F5527CA01880F991F880F4B
:10A71000991F880F991F9C01241B350BF901E25AE0
:10A72000F34F898184838A8185838B8186838C81A1
:10A7300080838D8181838E818283F901EF59F34F6C
:10A740008F81382F337088858370282F220F220F36
:10A75000888D982F9295907F822F832B892B8083D1
:10A76000FA01EC59F24F10821F5F143128F26896FB
:10A770000FB6F894DEBF0FBECDBFDF91CF911F9112
:10A7800008951F93CF93DF93CDB7DEB768970FB6C9
:10A79000F894DEBF0FBECDBF10E0A89519821A82D3
:10A7A0001B821C821D821E821F821886188E8FE0DB
:10A7B000189FC00111248858994FBC01CE010996F9
:10A7C0000E94C762BE016F5F7F4F812F0E9456318A
:10A7D0001F5F143110F368960FB6F894DEBF0FBEFA
:10A7E000CDBFDF91CF911F910895CF93C0E086E058
:10A7F000C89FC0011124FC01E451F34FF093EB0C0E
:10A80000E093EA0C80819181009719F00197918380
:10A810008083E091EA0CF091EB0C828193810097A8
:10A8200019F0019793838283E091EA0CF091EB0C8D
:10A8300084819581009719F00197958384832C2F4B
:10A840003327C901880F991F880F991F880F991FF7
:10A85000821B930BFC01E25AF34F8081882319F489
:10A860008181882321F08C2F8F5D0E944655CF5F18
:10A87000C43108F4BCCFCF91089599278730910552
:10A8800009F466C088309105ACF48430910509F470
:10A890003EC08530910534F48230910511F1039763
:10A8A00059F198C08530910509F43CC0069709F428
:10A8B00044C090C08A30910509F46BC08B3091057B
:10A8C00044F48830910509F44EC0099709F456C044
:10A8D00081C08B30910509F467C00C9709F46FC0F3
:10A8E00079C080EC0E94EC41882319F081E090E06F
:10A8F000089580E090E0089581EC0E94EC41882367
:10A9000019F081E090E0089580E090E0089582ECF5
:10A910000E94EC41882319F081E090E0089580E0E6
:10A9200090E0089581ED0E94EC41882319F081E0C8
:10A9300090E0089580E090E0089584EC0E94EC415E
:10A94000882319F081E090E0089580E090E0089578
:10A9500085EC0E94EC41882319F081E090E0089595
:10A9600080E090E0089586EC0E94EC41882319F085
:10A9700081E090E0089580E090E0089587EC0E94E7
:10A98000EC41882319F081E090E0089580E090E0A8
:10A99000089583EC0E94EC41882319F081E090E057
:10A9A000089580E090E0089582ED0E94EC418823B4
:10A9B00019F081E090E0089580E090E0089583ED43
:10A9C0000E94EC41882319F081E090E0089580E036
:10A9D00090E0089580E090E008950F93CF93DF9387
:10A9E000CDB7DEB721970FB6F894DEBF0FBECDBF4F
:10A9F00089838150843170F000E021E0AE014F5F27
:10AA00005F4F69E071E08FE891E00E94E92C80E0FF
:10AA100090E007C089819927FC01ED59F24F8081B0
:10AA2000992721960FB6F894DEBF0FBECDBFDF91F8
:10AA3000CF910F9108950F93CF93DF93CDB7DEB7EA
:10AA400021970FB6F894DEBF0FBECDBF8983843146
:10AA500060F000E021E0AE014F5F5F4F64E171E024
:10AA60008FE891E00E94E92C07C0898124E63DE04F
:10AA7000F901E80FF11D608321960FB6F894DEBF4F
:10AA80000FBECDBFDF91CF910F910895FF920F932D
:10AA90001F93CF93DF93CDB7DEB721970FB6F8940E
:10AAA000DEBF0FBECDBF1982813209F46DC0823284
:10AAB00019F481E0898368C0833219F482E08983C4
:10AAC00063C0843219F483E089835EC0853219F44F
:10AAD00084E0898359C0863219F485E0898354C0A3
:10AAE000873219F486E089834FC0883219F487E0F1
:10AAF00089834AC0893219F488E0898345C08A3243
:10AB000019F489E0898340C08B3219F48AE0898383
:10AB10003BC08C3219F48BE0898336C08D3219F436
:10AB20008CE0898331C08E3219F48DE089832CC08A
:10AB30008F3219F48EE0898327C0803319F48FE0B7
:10AB4000898322C0813319F480E189831DC0823357
:10AB500019F481E1898318C0833319F482E1898370
:10AB600013C0843319F483E189830EC000E021E02F
:10AB7000AE014F5F5F4F69E471E08FE891E00E94A2
:10AB8000E92C80E090E087C700E0102FF02E2981AB
:10AB900086E0289FC00111248451934F9093EB0CC1
:10ABA0008093EA0C3327C901880F991F880F991FDA
:10ABB000880F991F821B930BFC01E25AF34F80818F
:10ABC000882309F49BC18981282F3327C901880F65
:10ABD000991F880F991F880F991F821B930BFC01E7
:10ABE000E25AF34F80818F3F11F411E087C18981D0
:10ABF000282F3327C901880F991F880F991F880FA5
:10AC0000991F821B930BFC01E25AF34FE0818E2FB8
:10AC100082508B3008F04DC08E2F0E943D54482F3B
:10AC20008981282F3327C901880F991F880F991F01
:10AC3000880F991F821B930BFC01EF59F34F808102
:10AC400082958F7080FF02C081E04827442361F025
:10AC5000E091EA0CF091EB0C80819181892B11F449
:10AC600011E04CC110E04AC1A091EA0CB091EB0C8C
:10AC70008981282F3327C901880F991F880F991FB1
:10AC8000880F991F821B930BFC01E25AF34F9481AA
:10AC900085E0989FC00111248D939C93E091EA0C6C
:10ACA000F091EB0C8081918101969183808310E07B
:10ACB00025C18981282F3327C901880F991F880F43
:10ACC000991F880F991F821B930BFC01E25AF34FC7
:10ACD000E0818E2F8D50803208F04DC08F5F0E9432
:10ACE000E610482F8981282F3327C901880F991F23
:10ACF000880F991F880F991F821B930BFC01EF5936
:10AD0000F34F808182958F7080FF02C081E04827D9
:10AD1000442361F0E091EA0CF091EB0C8081918189
:10AD2000892B11F411E0EAC010E0E8C0A091EA0C10
:10AD3000B091EB0C8981282F3327C901880F991F07
:10AD4000880F991F880F991F821B930BFC01E25AF1
:10AD5000F34F948185E0989FC00111248D939C93BB
:10AD6000E091EA0CF091EB0C808191810196918346
:10AD7000808310E0C3C08981282F3327C901880F41
:10AD8000991F880F991F880F991F821B930BFC0135
:10AD9000E25AF34FE0818E2F8D52823208F04DC07F
:10ADA0008F5F0E946129482F8981282F3327C9018D
:10ADB000880F991F880F991F880F991F821B930B6B
:10ADC000FC01EF59F34F808182958F7080FF02C0A4
:10ADD00081E04827442361F0E091EA0CF091EB0C0C
:10ADE00080819181892B11F411E088C010E086C028
:10ADF000A091EA0CB091EB0C8981282F3327C9016F
:10AE0000880F991F880F991F880F991F821B930B1A
:10AE1000FC01E25AF34F948185E0989FC001112410
:10AE20008D939C93E091EA0CF091EB0C80819181E1
:10AE300001969183808310E061C08981282F332798
:10AE4000C901880F991F880F991F880F991F821BAE
:10AE5000930BFC01E25AF34FE0818E2F8F548F3019
:10AE600008F04CC08F5F0E94ED54482F8981282F35
:10AE70003327C901880F991F880F991F880F991FC1
:10AE8000821B930BFC01EF59F34F808182958F70E9
:10AE900080FF02C081E04827442361F0E091EA0C82
:10AEA000F091EB0C80819181892B11F411E026C087
:10AEB00010E024C0A091EA0CB091EB0C8981282FFE
:10AEC0003327C901880F991F880F991F880F991F71
:10AED000821B930BFC01E25AF34F948185E0989F0B
:10AEE000C00111248D939C93E091EA0CF091EB0C3E
:10AEF0008081918101969183808310E08981282F40
:10AF00003327C901880F991F880F991F880F991F30
:10AF1000821B930BFC01E25AF34F8181882311F4C9
:10AF2000082F9FC18981282F3327C901880F991FB6
:10AF3000880F991F880F991F821B930BFC01E25AFF
:10AF4000F34F81818F3F11F401E08BC18981282F5C
:10AF50003327C901880F991F880F991F880F991FE0
:10AF6000821B930BFC01E25AF34F9181892F82508F
:10AF70008B3008F04EC0892F0E943D54482F8981A4
:10AF8000282F3327C901880F991F880F991F880F11
:10AF9000991F821B930BFC01EF59F34F808182951F
:10AFA0008F7081FF02C081E04827442361F0E09167
:10AFB000EA0CF091EB0C82819381892B11F401E072
:10AFC00050C100E04EC1A091EA0CB091EB0C898118
:10AFD000282F3327C901880F991F880F991F880FC1
:10AFE000991F821B930BFC01E25AF34F958185E078
:10AFF000989FC0011124FD0193838283E091EA0CA4
:10B00000F091EB0C8281938101969383828300E01F
:10B0100028C18981282F3327C901880F991F880FDC
:10B02000991F880F991F821B930BFC01E25AF34F63
:10B030009181892F8D50803208F04EC08F5F0E9421
:10B04000E610482F8981282F3327C901880F991FBF
:10B05000880F991F880F991F821B930BFC01EF59D2
:10B06000F34F808182958F7081FF02C081E0482775
:10B07000442361F0E091EA0CF091EB0C8281938122
:10B08000892B11F401E0EDC000E0EBC0A091EA0CC7
:10B09000B091EB0C8981282F3327C901880F991FA4
:10B0A000880F991F880F991F821B930BFC01E25A8E
:10B0B000F34F958185E0989FC0011124FD01938392
:10B0C0008283E091EA0CF091EB0C828193810196EE
:10B0D0009383828300E0C5C08981282F3327C9016B
:10B0E000880F991F880F991F880F991F821B930B38
:10B0F000FC01E25AF34F9181892F8D52823208F080
:10B100004EC08F5F0E946129482F8981282F3327E5
:10B11000C901880F991F880F991F880F991F821BDB
:10B12000930BFC01EF59F34F808182958F7081FF63
:10B1300002C081E04827442361F0E091EA0CF091DD
:10B14000EB0C82819381892B11F401E08AC000E02D
:10B1500088C0A091EA0CB091EB0C8981282F33278D
:10B16000C901880F991F880F991F880F991F821B8B
:10B17000930BFC01E25AF34F958185E0989FC00143
:10B180001124FD0193838283E091EA0CF091EB0C92
:10B190008281938101969383828300E062C08981DA
:10B1A000282F3327C901880F991F880F991F880FEF
:10B1B000991F821B930BFC01E25AF34F9181892F57
:10B1C0008F548F3008F04DC08F5F0E94ED54482F90
:10B1D0008981282F3327C901880F991F880F991F4C
:10B1E000880F991F821B930BFC01EF59F34F80814D
:10B1F00082958F7081FF02C081E04827442361F06F
:10B20000E091EA0CF091EB0C82819381892B11F48F
:10B2100001E027C000E025C0A091EA0CB091EB0C42
:10B220008981282F3327C901880F991F880F991FFB
:10B23000880F991F821B930BFC01E25AF34F9581F3
:10B2400085E0989FC0011124FD0193838283E091E2
:10B25000EA0CF091EB0C82819381019693838283B7
:10B2600000E08981282F3327C901880F991F880F93
:10B27000991F880F991F821B930BFC01E25AF34F11
:10B280008281882311F4F82EA4C18981282F3327C5
:10B29000C901880F991F880F991F880F991F821B5A
:10B2A000930BFC01E25AF34F82818F3F19F4FF2484
:10B2B000F3948FC18981282F3327C901880F991FE3
:10B2C000880F991F880F991F821B930BFC01E25A6C
:10B2D000F34F9281892F82508B3008F04FC0892F15
:10B2E0000E943D54482F8981282F3327C901880F98
:10B2F000991F880F991F880F991F821B930BFC01C0
:10B30000EF59F34F808182958F7082FF02C081E0F8
:10B310004827442369F0E091EA0CF091EB0C84811A
:10B320009581892B19F4FF24F39453C1FF2451C153
:10B33000A091EA0CB091EB0C8981282F3327C90129
:10B34000880F991F880F991F880F991F821B930BD5
:10B35000FC01E25AF34F968185E0989FC0011124C9
:10B36000FD0195838483E091EA0CF091EB0C8481DC
:10B370009581019695838483FF242BC18981282F91
:10B380003327C901880F991F880F991F880F991FAC
:10B39000821B930BFC01E25AF34F9281892F8D504F
:10B3A000803208F04FC08F5F0E94E610482F8981DD
:10B3B000282F3327C901880F991F880F991F880FDD
:10B3C000991F821B930BFC01EF59F34F80818295EB
:10B3D0008F7082FF02C081E04827442369F0E0912A
:10B3E000EA0CF091EB0C84819581892B19F4FF24F0
:10B3F000F394EFC0FF24EDC0A091EA0CB091EB0CE8
:10B400008981282F3327C901880F991F880F991F19
:10B41000880F991F821B930BFC01E25AF34F968110
:10B4200085E0989FC0011124FD0195838483E091FC
:10B43000EA0CF091EB0C84819581019695838483CD
:10B44000FF24C7C08981282F3327C901880F991F7E
:10B45000880F991F880F991F821B930BFC01E25ADA
:10B46000F34F9281892F8D52823208F04FC08F5F47
:10B470000E946129482F8981282F3327C901880F0D
:10B48000991F880F991F880F991F821B930BFC012E
:10B49000EF59F34F808182958F7082FF02C081E067
:10B4A0004827442369F0E091EA0CF091EB0C848189
:10B4B0009581892B19F4FF24F3948BC0FF2489C054
:10B4C000A091EA0CB091EB0C8981282F3327C90198
:10B4D000880F991F880F991F880F991F821B930B44
:10B4E000FC01E25AF34F968185E0989FC001112438
:10B4F000FD0195838483E091EA0CF091EB0C84814B
:10B500009581019695838483FF2463C08981282FC8
:10B510003327C901880F991F880F991F880F991F1A
:10B52000821B930BFC01E25AF34F9281892F8F54B7
:10B530008F3008F04EC08F5F0E94ED54482F8981F4
:10B54000282F3327C901880F991F880F991F880F4B
:10B55000991F821B930BFC01EF59F34F8081829559
:10B560008F7082FF02C081E04827442369F0E09198
:10B57000EA0CF091EB0C84819581892B19F4FF245E
:10B58000F39427C0FF2425C0A091EA0CB091EB0CE6
:10B590008981282F3327C901880F991F880F991F88
:10B5A000880F991F821B930BFC01E25AF34F96817F
:10B5B00085E0989FC0011124FD0195838483E0916B
:10B5C000EA0CF091EB0C848195810196958384833C
:10B5D000FF242981822F9927AC01440F551F440F66
:10B5E000551F440F551F481B590BDA01A25AB34F80
:10B5F0008C91882309F47FC1FD018181882309F49E
:10B600007AC18281882309F476C1FA01EF59F34F98
:10B61000E0818E2F837009F084C0112309F43EC0AD
:10B620000023E1F18E2F86958695837061F46F2D4E
:10B63000822F0E941B55FF2019F081E090E02BC261
:10B6400080E090E028C28981282F3327C901880F24
:10B65000991F880F991F880F991F821B930BFC015C
:10B66000EF59F34F8081869586958370823079F407
:10B6700060E01F1509F461E089810E941B551F15C8
:10B6800019F481E090E007C280E090E004C261E03C
:10B6900089810E941B5581E090E0FDC14981242FE2
:10B6A0003327C901880F991F880F991F880F991F89
:10B6B000821B930BFC01EF59F34F80818695869591
:10B6C0008370823049F4FF2039F461E0842F0E94B6
:10B6D0001B5581E090E0DFC14981242F3327C90148
:10B6E000880F991F880F991F880F991F821B930B32
:10B6F000FC01EF59F34F808186958695682F637022
:10B70000613041F4FF2031F0842F0E941B5581E00D
:10B7100090E0C1C160E089810E941B5580E090E00B
:10B72000BAC14981242F3327C901880F991F880F77
:10B73000991F880F991F821B930BFC01EF59F34F40
:10B74000E0818E2F8370823009F045C01017E1F53B
:10B750008E2F86958695837061F46F2D842F0E94BD
:10B760001B55FF2019F081E090E095C180E090E04A
:10B7700092C18981282F3327C901880F991F880F0B
:10B78000991F880F991F821B930BFC01EF59F34FF0
:10B790008081869586958370823079F460E01F15EC
:10B7A00009F461E089810E941B551F1519F481E09D
:10B7B00090E071C180E090E06EC161E089810E94FB
:10B7C0001B5581E090E067C160E089810E941B55B4
:10B7D00080E090E060C1112319F4002309F448C00F
:10B7E0004981242F3327C901880F991F880F991F7A
:10B7F000880F991F821B930BFC01EF59F34F808137
:10B8000086958695837061F46F2D842F0E941B5559
:10B81000FF2019F081E090E03EC180E090E03BC164
:10B820004981242F3327C901880F991F880F991F39
:10B83000880F991F821B930BFC01EF59F34F8081F6
:10B84000869586958370823061F46F2D842F0E94D7
:10B850001B55FF2019F081E090E01DC180E090E0D1
:10B860001AC161E089810E941B5581E090E013C1FB
:10B870004981242F3327C901880F991F880F991FE9
:10B88000880F991F821B930BFC01EF59F34F8081A6
:10B8900086958695682F6370613041F4FF2021F111
:10B8A000842F0E941B5581E090E0F5C04981242F30
:10B8B0003327C901880F991F880F991F880F991F77
:10B8C000821B930BFC01EF59F34F8081869586957F
:10B8D0008370823049F4FF2039F461E0842F0E94A4
:10B8E0001B5581E090E0D7C060E089810E941B5524
:10B8F00080E090E0D0C02981822F9927AC01440FCD
:10B90000551F440F551F440F551F481B590BDA0193
:10B91000A25AB34F8C91882309F452C0FD01818152
:10B92000882309F44DC0FA01EF59F34F80818370E9
:10B9300091F4112349F0002339F061E0822F0E9435
:10B940001B5581E090E0A7C060E089810E941B55F3
:10B9500080E090E0A0C04981242F3327C901880FDF
:10B96000991F880F991F880F991F821B930BFC0149
:10B97000EF59F34F80818370823081F4101739F4CE
:10B9800061E0842F0E941B5581E090E084C060E05C
:10B9900089810E941B5580E090E07DC0112311F445
:10B9A000002339F061E089810E941B5581E090E01D
:10B9B00072C060E089810E941B5580E090E06BC0FE
:10B9C0002981822F9927AC01440F551F440F551F21
:10B9D000440F551F481B590BDA01A25AB34FFD0102
:10B9E0008181882309F455C08281882309F451C0DC
:10B9F000FA01EF59F34F808186958695837091F413
:10BA0000112349F0002339F061E0822F0E941B5579
:10BA100081E090E040C060E089810E941B5580E099
:10BA200090E039C04981242F3327C901880F991F1D
:10BA3000880F991F880F991F821B930BFC01EF59E8
:10BA4000F34F8081869586958370823081F410173C
:10BA500039F461E0842F0E941B5581E090E01BC007
:10BA600060E089810E941B5580E090E014C01123A2
:10BA700011F4002339F061E089810E941B5581E0B7
:10BA800090E009C060E089810E941B5580E090E051
:10BA900002C080E090E021960FB6F894DEBF0FBEA2
:10BAA000CDBFDF91CF911F910F91FF900895CF935C
:10BAB000DF93CDB7DEB721970FB6F894DEBF0FBE88
:10BAC000CDBF282F04B603FE28C0FE013196ACEB93
:10BAD000B0E081E090E031E08030930719F40E94FB
:10BAE000C76303C0182E0E94C7638981843190F414
:10BAF0008F5F8983FE013196ACEBB0E081E090E08E
:10BB000031E08030930719F40E94D86303C0182EE7
:10BB10000E94D86384B7877F84BF8091600088616A
:10BB20008093600020936000809160008860809323
:10BB3000600021960FB6F894DEBF0FBECDBFDF9137
:10BB4000CF910895EF92FF920F931F937B018C0189
:10BB500020E030E040E05FE40E94066088239CF033
:10BB600020E030E040E05FECC801B7010E94F05EE9
:10BB7000DC01CB01BC01CD010E94A060605070408F
:10BB80008040904804C0C801B7010E94A0601F9186
:10BB90000F91FF90EF900895A0E0B0E0E2EDFDE599
:10BBA0000C9488638C017B015A01DC018C918230FA
:10BBB00058F0FB019081923010F4A7010BC1843042
:10BBC00029F4943009F4A6C0A80104C19430A9F363
:10BBD000923009F4A9C0823081F3F801C280D38089
:10BBE000FB0162817381F80124813581468157818F
:10BBF000F7016480758086809780C601861B970B4D
:10BC000097FDD8C080970CF46CC06C157D050CF0C6
:10BC1000ADC0662477244301F8016181F701818179
:10BC2000681709F499C0662309F491C0621A730A6F
:10BC3000840A950AA401930157FDC0C0F501118241
:10BC4000B60119012A0179018A0139014A010894D2
:10BC50006108710881089108FFEF6F16FFEF7F06FA
:10BC6000FFEF8F06FFE39F06F0F4A8019701220F74
:10BC7000331F441F551F19012A01B601615070403E
:10BC80006B0179018A0139014A0108946108710840
:10BC9000810891088FEF68168FEF78068FEF88067E
:10BCA0008FE3980610F383E0D5018C9357FC64C0B2
:10BCB000F501248335834683578373836283A5010B
:10BCC00089C06F5F7F4FD401C30181709070A070F5
:10BCD000B0709694879477946794682A792A8A2A10
:10BCE0009B2A6C157D056CF311C00894C11CD11CF6
:10BCF000DA01C90181709070A070B07056954795B7
:10BD000037952795282B392B4A2B5B2BC616D70640
:10BD100064F382CFF8019181FB018181981709F4C6
:10BD200053CF42EA51E056C0823009F04DCF88E04F
:10BD3000DA01F80101900D928A95E1F7F80181810D
:10BD4000FB0191818923FA018183A50143C0261952
:10BD500037094809590970CFF5016183B601260DED
:10BD6000371D481D591D19012A019DCF6B0120E087
:10BD700030E040E050E050CFD201C101B695A79528
:10BD80009795879521E030E040E050E02222332271
:10BD900044225522282A392A4A2A5B2AF50124827C
:10BDA0003582468257820894C11CD11CD382C2823C
:10BDB000A50110C0909581959F4F24CF81E0F5019A
:10BDC0008183B60150954095309521953F4F4F4F57
:10BDD0005F4F37CFCA01E2E1CDB7DEB70C94A46361
:10BDE000A0E2B0E0E6EFFEE50C949663DC01CB0147
:10BDF000898F9A8FAB8FBC8F2D8F3E8F4F8F58A31B
:10BE0000BE016F5F7F4FCE0149960E94DA618E01BD
:10BE1000075F1F4FB801CE014D960E94DA61AE0157
:10BE20004F5E5F4FB801CE0101960E94CC5D0E942B
:10BE3000F260DC01CB01BC01CD01E4E0A0960C94E2
:10BE4000B263A0E2B0E0E7E2FFE50C949663DC01A8
:10BE5000CB01898F9A8FAB8FBC8F2D8F3E8F4F8FE9
:10BE600058A3BE016F5F7F4FCE0149960E94DA61F1
:10BE70008E01075F1F4FB801CE014D960E94DA6117
:10BE80008A8591E089278A87AE014F5E5F4FB801AE
:10BE9000CE0101960E94CC5D0E94F260DC01CB01D4
:10BEA000BC01CD01E4E0A0960C94B263A8E1B0E03F
:10BEB000ECE5FFE50C949063DC01CB01898B9A8B58
:10BEC000AB8BBC8B2D8B3E8B4F8B588FBE016F5F26
:10BED0007F4FCE0141960E94DA618E01075F1F4FAE
:10BEE000B801CE0145960E94DA61FE0131962981A2
:10BEF000223008F45FC03985323010F4B8017BC0BD
:10BF000081819A8589278183243009F455C02230A4
:10BF100009F452C0343009F454C0323009F458C026
:10BF20006B817C818B859C85681B790B2D813E8183
:10BF30004F815885ED84FE840F8518892E153F05A5
:10BF40004007510730F4220F331F441F551F615023
:10BF500070407C836B8380E090E0A0E0B0E4AA2492
:10BF6000BB2465012E153F054007510740F0A82A64
:10BF7000B92ACA2ADB2A2E193F09400B510BB69564
:10BF8000A79597958795220F331F441F551F00973C
:10BF9000A105B10539F7D601C5018F779070A07062
:10BFA000B07080349105A105B105A9F0A482B582D5
:10BFB000C682D782BF011FC02317E1F762EA71E092
:10BFC0001AC01D821E821F8218861C821B82F2CF1D
:10BFD00084E08983EFCFA7FC05C021153105410519
:10BFE000510521F380E490E0A0E0B0E0A80EB91E76
:10BFF000CA1EDB1EDBCFCB010E94F260DC01CB014D
:10C00000BC01CD01EAE068960C94AC63A8E1B0E015
:10C01000ECE0F0E60C949663DC01CB01898B9A8B03
:10C02000AB8BBC8B2D8B3E8B4F8B588FBE016F5FC4
:10C030007F4FCE0141960E94DA618E01075F1F4F4C
:10C04000B801CE0145960E94DA618981823018F0EC
:10C050008985823018F42FEF3FEF09C0B801CE0177
:10C0600001960E945462282F332727FD3095C9017D
:10C07000E4E068960C94B263A8E0B0E0E2E4F0E695
:10C080000C9494639B01AC017B018C01EE2417FDA1
:10C09000E394FF2400271127EA8221153105410589
:10C0A000510539F482E08983CE0101960E94F26045
:10C0B00043C083E089836EE170E0CB01EE2031F56F
:10C0C00079018A01A80197012030E0E03E07E0E015
:10C0D0004E07E0E45E0798F479018A01EE0CFF1C3C
:10C0E000001F111F0197BC01A8019701E0E0EE16A7
:10C0F000E0E0FE06E0E00E07E0E41E0768F3ED82F4
:10C10000FE820F8318877C836B83CECF2030E0E0E4
:10C110003E07E0E04E07E0E85E0741F0EE24FF2432
:10C120008701E21AF30A040B150BCCCF7C836B83D7
:10C1300060E070E080E09FECE6E028960C94B0634D
:10C14000ACE0B0E0E6EAF0E60C949863DC01CB01E9
:10C1500089879A87AB87BC87BE016F5F7F4FCE010F
:10C1600009960E94DA618981823011F0823028F4C8
:10C1700060E070E080E090E031C0843039F02B81E5
:10C180003C8137FDF5CF2F3131056CF08A81882352
:10C1900029F060E070E080E090E820C06FEF7FEF72
:10C1A0008FEF9FE71BC08EE190E0821B930B2D81E8
:10C1B0003E814F81588504C0569547953795279500
:10C1C0008A95D2F78A81882339F050954095309529
:10C1D00021953F4F4F4F5F4FCA01B901E2E02C96C6
:10C1E0000C94B463A0E0B0E0E8EFF0E60C948E634A
:10C1F000882499245401DC01FC0124813581468185
:10C2000057818181082F112760E070E08C91823086
:10C2100020F46FEF70E04061A4C0843009F464C082
:10C22000823009F463C0211531054105510509F437
:10C2300098C0FD0182819381FFEF82389F070CF047
:10C2400050C0A2E8EA2EAFEFFA2EE81AF90A8AE106
:10C25000E816F1040CF06BC06B0181E090E0A0E007
:10C26000B0E00E2C04C0880F991FAA1FBB1F0A94B0
:10C27000D2F70197A109B10982239323A423B523FF
:10C280000097A105B10519F0F1E0CF2ED12C04C023
:10C290005695479537952795EA94D2F7C601AA2770
:10C2A00097FDA095BA2F282B392B4A2B5B2BDA014F
:10C2B000C9018F779070A070B07080349105A1058E
:10C2C000B105D1F1215C3F4F4F4F5F4F2030E0E08F
:10C2D0003E07E0E04E07E0E45E0708F161E070E051
:10C2E0001EC0803891053CF06FEF70E020E030E038
:10C2F00040E050E036C0BC0161587F4FDA01C9010F
:10C300008F779070A070B07080349105A105B10551
:10C31000D1F0215C3F4F4F4F5F4F57FD1BC097E05F
:10C3200056954795379527959A95D1F71AC020E0ED
:10C3300030E040E050E0BBCF27FFC8CF205C3F4F4C
:10C340004F4F5F4FC3CF27FFE8CF205C3F4F4F4F8A
:10C350005F4FE3CF56954795379527956F5F7F4F92
:10C36000DECF822E932E942F9F778A2D8078A82E51
:10C37000A92A962F9795992797958A2D8F77A82E7A
:10C38000A92A76956795962F9F778B2D8078B82E62
:10C39000B92A902F9795992797958B2D8F77B82E3F
:10C3A000B92AD501C401BC01CD01ECE0CDB7DEB79F
:10C3B0000C94AA63CF93DF93FC01DB014081518190
:10C3C0002281622F6F7770E0221F2227221F938124
:10C3D000892F880F822B282F3327991F9927991F80
:10C3E000ED0199832115310541F441155105610590
:10C3F0007105E1F482E08C9354C02F3F310509F4BC
:10C4000041C02F573040FD013383228383E08C935A
:10C4100087E0440F551F661F771F8A95D1F7706418
:10C42000ED014C835D836E837F833BC022E83FEF49
:10C43000F901C7E0440F551F661F771FCA95D1F752
:10C4400083E08C93403080E0580780E0680780E408
:10C45000780778F4440F551F661F771F215030402E
:10C46000F9014030C0E05C07C0E06C07C0E47C0725
:10C4700088F3ED01FB83EA83FD01448355836683E2
:10C4800077830FC0411551056105710519F484E0EA
:10C490008C9307C064FF03C081E08C93C1CF1C92D2
:10C4A000BFCFDF91CF9108950F931F93CF93DF9369
:10C4B000FC01DB018081823018F09C91923018F4ED
:10C4C00061E070E05EC08430C1F0843001F19430EE
:10C4D00009F447C0823009F44BC0823009F44EC0E1
:10C4E0009230A9F04181ED0189814817B9F04423C8
:10C4F00089F08FEF9FEFBC0144C0943031F7EB011E
:10C500008981682F77278181681B71093AC08181F1
:10C51000882379F781E090E0BC0133C02281338128
:10C52000ED018A819B81821793070CF32817390745
:10C530009CF00481158126813781FD01648175811C
:10C5400086819781601771078207930780F206172B
:10C5500017072807390778F4442359F281E090E05F
:10C56000DBCFFD018181882321F281E090E0D4CFEF
:10C57000923009F0B2CF60E070E003C0ED01898134
:10C58000F2CFCB01DF91CF911F910F910895FB0165
:10C59000DC0105900D920020E1F70895FB01DC011C
:10C5A00004C08D910190801921F441505040C8F78A
:10C5B000881B990B0895FB01DC0140FF05C002C0F8
:10C5C00001900D9201900D9242505040C8F708958D
:10C5D000DC0140FF03C001C06D936D934250504099
:10C5E000D8F70895FB01DC0101900D920020E1F7DE
:10C5F0000895629FD001739FF001829FE00DF11DAD
:10C60000649FE00DF11D929FF00D839FF00D749FCC
:10C61000F00D659FF00D9927729FB00DE11DF91F78
:10C62000639FB00DE11DF91FBD01CF0111240895D5
:10C63000991B79E004C0991F961708F0961B881F74
:10C640007A95C9F780950895AA1BBB1B51E107C0D5
:10C65000AA1FBB1FA617B70710F0A61BB70B881F92
:10C66000991F5A95A9F780959095BC01CD01089521
:10C6700097FB092E07260AD077FD04D0E5DF06D008
:10C6800000201AF4709561957F4F0895F6F7909504
:10C6900081959F4F0895A1E21A2EAA1BBB1BFD0195
:10C6A0000DC0AA1FBB1FEE1FFF1FA217B307E40791
:10C6B000F50720F0A21BB30BE40BF50B661F771FE9
:10C6C000881F991F1A9469F76095709580959095C9
:10C6D0009B01AC01BD01CF01089597FB092E0526F2
:10C6E0000ED057FD04D0D7DF0AD0001C38F4509587
:10C6F0004095309521953F4F4F4F5F4F0895F6F786
:10C7000090958095709561957F4F8F4F9F4F0895BD
:10C710002F923F924F925F926F927F928F929F9251
:10C72000AF92BF92CF92DF92EF92FF920F931F933F
:10C73000CF93DF93CDB7DEB7CA1BDB0B0FB6F894F0
:10C74000DEBF0FBECDBF09942A88398848885F8430
:10C750006E847D848C849B84AA84B984C884DF80A1
:10C76000EE80FD800C811B81AA81B981CE0FD11D85
:10C770000FB6F894DEBF0FBECDBFED010895F99955
:10C78000FECFB2BDA1BDF89A119600B40895F7DFAF
:10C7900001921A94E1F70895F999FECFB2BDA1BDB7
:10C7A00000BC11960FB6F894FA9AF99A0FBE089544
:0AC7B0000190F2DF1A94E1F70895FA
:10C7BA0001012E2E2F63616E5F696E7075742E6390
:10C7CA00006E222E2E2F6368616E6E656C732E6367
:10C7DA000053657175656E63652023310053657179
:10C7EA0075656E63652023320053657175656E63E6
:10C7FA00652023330053657175656E6365202334A4
:10C80A0000455233002E2E2F656570726F6D636876
:10C81A00616E6E656C732E630050434D3000455255
:10C82A0033004C4F4730340050434D207665722018
:10C83A00392E3134004F425220383434300B002E16
:10C84A002E2F7669727475656C5F696E7075742EB9
:0AC85A006300000000000000000071
:00000001FF
